:020000040000FA
:040000009EEF14F06B
:08000800DDEF14F0186E7F0B10
:1000100018BC8008F76A240FF66E0800F55018BE69
:1000200000081200000306090C101316191C1F22E9
:1000300025282B2E313336393C3F414447494C4E1D
:10004000515355585A5C5E60626466686A6B6D6FA6
:1000500070717374757678797A7A7B7C7D7D7E7E1B
:100060007E7F7F7F7F002C6A2D6A01D0206E215019
:10007000205ED8A021062D502C5ED8A02D06D89049
:1000800021322032D8902D322C32031C1C6E041CDD
:100090001D6E1C2AD8B41D2A830E276E286A296A71
:1000A0002A6A2B6A266A0F0EEA6E02C0E9FF091C53
:1000B000D5EC02F000D000D0040020502826D8B0A3
:1000C000292A215029262C502A26D8B02B2A2D50F7
:1000D0002B2629509BDF800F196E2B5097DF800F46
:1000E00019261930262602C0E9FFEF500910D8A0C2
:1000F0000918EF6E2704D8B4830E276ED8B41C2AD3
:10010000D8B41D3ED7D71200086A800E346E89EF2E
:1001100000F0206A216A226A236A0A9AF2EC01F04E
:10012000D30FD8B40A8A2D0FC60FF8E20A0FF6E3F0
:100130001C6E1B6A1A6A196A0A0E186EB3EC02F07A
:100140001C501824206E1950216E000ED8B0010EDC
:1001500021261A50226E000ED8B0010E22261B5006
:10016000236E000ED8B0010E2326080606E0F2EC3E
:1001700001F0C60F02E20A0FDBE20AAA0BD0201E32
:10018000211E221E231E202AD8B4212AD8B4222AB6
:10019000D8B4232A20501200086A206E216A0096E3
:1001A0000850D8B40086050E076E270E1D6E100E7F
:1001B0000CD8030E1D6EE80E08D81D6A640E05D813
:1001C0001D6A0A0E02D8205008D01C6E2150196EEC
:1001D0002050186E9CEC02F01850186E074E0096D6
:1001E000085003E0075CD8B008D01850D8A4009697
:1001F00000B603D0300FE5EF01F01200366E2DAEE1
:1002000003D02D0EE5EC01F0106A116A126A136A30
:100210002D8E6A0E2C26D8902D322E322F3213328C
:100220001232113210322C3EF6D72F502C5C2F2672
:100230002C5E2E502D5C2E262D5E086A3AD82E0E8E
:10024000E5EC01F0376AD89010342F6E11342E6E21
:1002500012342D6E13342C6E3736D8902F362E363E
:100260002D362C36373610502F261150D8B0113C71
:100270002E261250D8B0123C2D261350D8B0133C65
:100280002C26D8B0373ED8902F362E362D362C3629
:1002900037363750300FE5EC01F02FC010F02EC08C
:1002A00011F02DC012F02CC013F0362ECBD7D89001
:1002B00012000096085003E100860A0E086E2FC057
:1002C0001BF02EC01AF02DC019F02CC018F0076AD0
:1002D000236A226A216A0A0E206E3FEC02F0072A86
:1002E0000750085CD8A4F4D72050D8A4009600A6E4
:1002F00002D0082C04D02050300FE5EC01F0082E7D
:10030000DED71200206E0750D8B4120020C0E9FFDB
:1003100021C0EAFFEF50D8B41200E5EC01F0204A0A
:10032000212A0706F0D7246E0F0EEA6EE26E025005
:10033000E96E120FE16E800E0A16080E256ED89037
:10034000D8B00A3E12D82432252EFAD7000029BA96
:100350000A300BD800D000D000D0D88006D8065084
:100360001D6E055025EC02F0120029AE0BD0EF50A7
:10037000091029AC0918EF6EE7500910D8A0091828
:10038000E76E0AD0EF500910D8A0091829BC091847
:10039000EF6E091CE71600D029501F0B000F196ED5
:1003A0002850110FD8B0192A000032EF02F0A66AC7
:1003B000A68E0900F55002E002D8FBD71200040017
:1003C0009EA8FDD7AD6ED880120001BA93EF01F060
:1003D00001B4DFEF01F001A205D001B003D001B2FA
:1003E000EE6E120034BEEE501200AA6AA96EA66A22
:1003F000A680A850A94AAA2A1200AA6AA86EA66ACC
:10040000A684550EA76EAA0EA76EA6820400A6B2F9
:10041000FDD7A694A94AAA2A1200E836E8363C0B72
:100420000109C212C009C216C050F80B0209C06E01
:10043000320E31EC02F0C2820400C2B2FDD7C4CF4A
:100440002DF0C3502C6E12001D6A1C6EFF0E1C2670
:100450001D2200D0D8A01200030E196EE70E02D89C
:10046000F5D7196AFD0F186EFF0E00D001D01826BF
:10047000040000D0D8A01926D8A01200F8D71B502D
:100480002318800BF46E1BAE06D0D880000E1856D1
:1004900019561A561B5623AE06D0D880000E205689
:1004A0002156225623561C6A1D6A1E6A1F6A306A2C
:1004B000316A326A336A235022102110201023E05F
:1004C000200EF36ED890183619361A361B36303691
:1004D0003136323633362050305C2150315822507C
:1004E00032582350335809E32050305E2150315A9E
:1004F0002250325A2350335AD8801C361D361E36AD
:100500001F36F32EDFD7F4AE06D0D880000E1C566F
:100510001D561E561F561CC018F01DC019F01EC0D7
:100520001AF01FC01BF030C020F031C021F032C0E3
:1005300022F033C023F01200216A206A100EF36EFD
:100540001934203621361C50205C1D50215805E3FB
:100550001C50205E1D50215AD88018361936F32EB3
:10056000EFD718501200200E246E306A316A326ABA
:10057000336AD89018A00ED0205030262150D8B021
:10058000213C31262250D8B0223C32262350D8B00C
:10059000233C332633323232313230321B321A327C
:1005A00019321832242EE5D71200E988E92AEC1610
:1005B0001200A66AA68E0900F55002E0EE6EFBD787
:1005C0001200F34E02D0E652FCD7E6CFEEFFE82E43
:1005D000FCD71200E466FED7F36EE552F32EFDD78A
:1005E000E6CFEEFFE82EFCD71200610EE75C05E6D1
:1005F0007B0EE75C02E7DF0EE716E650EE6EF5E1F4
:100600001200A66AA68EEE500900F55C02E1F566BE
:10061000FAD71200155011183A6E3ABE30D015BEF6
:1006200017D01450105CD8A0000CD8A4010C1550A1
:10063000115CD8A0000CD8A4010C1650125CD8A0F4
:10064000000CD8A4010C1750135CD8A0000C010CAE
:100650001050145CD8A0000CD8A4010C1150155CEB
:10066000D8A0000CD8A4010C1250165CD8A0000C25
:10067000D8A4010C1350175CD8A0000C010C11AECB
:10068000010C000C155011183A6E3ABE34D015BE4C
:1006900019D01450105CD8A0000CD8A4010C15502F
:1006A000115CD8A0000CD8A4010C1650125CD8A084
:1006B000000CD8A4010C1750135CD8A0000CD8A4CF
:1006C000010C000C1050145CD8A0000CD8A4010C34
:1006D0001150155CD8A0000CD8A4010C1250165C67
:1006E000D8A0000CD8A4010C1350175CD8A0000CA3
:1006F000D8A4010C000C11AE010C000C1450105CBD
:10070000376E19E2376C10C039F014C010F039C0E0
:1007100014F011C039F015C011F039C015F012C035
:1007200039F016C012F039C016F013C039F017C0F6
:1007300013F039C017F01A0E376078D0145276E0F3
:10074000366A1150396E15183B6E118E158E080ED3
:10075000375E08E317C036F016C017F015C016F064
:10076000156AF5D7372607E0D890153216321732BA
:100770003632372EF9D73BAE35D01750135E1650B0
:10078000125A1550115A07E2D880000E135612560D
:100790001156800E391A366C04E01306000E125AF8
:1007A000115A040E376E11660DD012C011F013C02D
:1007B00012F036C013F0366A080E105E2DE3372EA5
:1007C000F2D72AD011BE08D0D8903636133612365A
:1007D0001136102EF7D720D038AC26D036AE24D024
:1007E000366A11D0175013261650122215501122B6
:1007F00006E31132123213323632104A0FD038ACBF
:1008000013D036AE11D0133E0FD0123E0DD0113E94
:100810000BD0D8801390EDD7106A02D038821068C0
:10082000136A126A800E116E39AE119E13501200B7
:100830001150326E15183B6E145053E0105254E0B4
:10084000105E7F0E03E2102603E24DD010264EE22A
:1008500013C030F012C031F0328E158E180E396E82
:10086000136A126A116A0BD01750305C1650315857
:1008700011E3316E326A1750305E0BD004E215502E
:10088000325CF2E007E31750305E1650315A1550D3
:10089000325AD88013361236113630363136323667
:1008A000392EECD711BE07D010521DE03B32100696
:1008B000392A3B36E3D738AC1FD007E21750305EF9
:1008C0001650315A1550325A17E3133E15D0123EC6
:1008D00013D0113E11D0113212321332103E0CD00F
:1008E00005D0388604D03884106A02D03882106867
:1008F000136A126A800E116E3BAE119E13501200E5
:100900001150326E15183B6E1050D8A414503CE0B4
:1009100010267E0E03E3105E03E338D0105E33E34F
:1009200013C030F012C031F0328E158E136A126A85
:10093000116A180E396E32323132303206E31750F6
:100940001326165012221550112211321232133270
:10095000392EF1D711BE07D0133612361136105288
:1009600012E01006323438AC17D016E3133E14D020
:10097000123E12D0113E10D0D880113212321332F2
:10098000103E0AD003D03884106A02D03882106832
:10099000136A126A800E116E3BAE119E1350120044
:1009A000126A136A10C036F013C010F036C013F08C
:1009B00012C036F011C012F036C011F0960E396E2A
:1009C0003B6A10AE07D0D880000E1356125611564F
:1009D00010563B8E105218E038AC0DD013AE0BD031
:1009E000123E09D0113E07D0103E05D0D8801032FB
:1009F00011321232392A080E392612C013F011C0F2
:100A000012F010C011F015D0116613D0080E395E27
:100A1000125005E1080E395E135011E0136A116E91
:100A200013C012F0136A05D0D8901336123611365F
:100A3000390611AEF9D739C010F03BAE119E1350F4
:100A400012003D3D3D3D3D3D3D3D3D3D3D3D3D3D3E
:100A50003D3D3D3D3D3D3D3D3D3D3D3D3D3D3D3DC6
:100A60003D3D3D3D3D3D3D3D3D004E657720435084
:100A70005520636869702064657465637465642ECD
:100A800000003D3D3D3D3D3D3D3D3D3D3D3D3D3D10
:100A90003D3D3D3D3D3D3D3D3D3D3D3D3D3D3D3D86
:100AA0003D3D3D3D3D3D3D3D3D003D3D3D3D3D3DB3
:100AB0003D3D3D3D3D3D3D3D3D3D3D3D3D3D3D3D66
:100AC0003D3D3D3D3D3D3D3D3D3D3D3D3D3D3D3D56
:100AD0003D0053696572726120526164696F2053F1
:100AE000797374656D732054522053657175656E0A
:100AF000636572004669726D776172652076657212
:100B000073696F6E20002C206275696C6420000090
:100B10004E6574776F726B206164647265737320C5
:100B20002000456E746572202F2F68656C702066FA
:100B30006F7220636F6D6D616E642073756D6D6192
:100B4000727900003D3D3D3D3D3D3D3D3D3D3D3DDE
:100B50003D3D3D3D3D3D3D3D3D3D3D3D3D3D3D3DC5
:100B60003D3D3D3D3D3D3D3D3D3D3D00456E74655A
:100B70007220636F6D6D616E642000002F2F6F75A2
:100B8000743033206F6E00004641494C00004865C8
:100B90007921206E657720636F6D6D616E64000052
:100BA0006E65745F7061636B65742073686F756CDC
:100BB0006420626520636C656172203C00006E6594
:100BC000745F7061636B65745F6C656E203D2000BF
:100BD0007061636B6574203D20006E65745F73798E
:100BE0006E633D006E65745F747970653D006E657F
:100BF000745F66726F6D3D006E65745F746F3D006B
:100C00006E65745F6372633D00006E65745F706152
:100C1000796C6F61643D3C006E65745F7061636BFD
:100C200065745F6C656E3D006E65745F7061796CB4
:100C30006F61645F6C656E3D00002E2E2E20636830
:100C400065636B2074686520435243202E2E2E006E
:100C50006C656E677468206F6620617267203D2046
:100C6000000043616C63756C61746564204352439A
:100C7000203D20002C205061636B6574204352435B
:100C8000203D2000435243204661696C65642E205C
:100C900020426164207061636B657400435243209D
:100CA00050617373656420212020476F6F6420506A
:100CB00061636B6574006D79206164647265737340
:100CC0003D00484559212074686973207061636B49
:100CD000657420697320666F72206D6521004E6F08
:100CE00074206D79206164647265737300005365CC
:100CF0006E643A20000053656E643A20000053652C
:100D00006E643A20000053656E643A20000049206A
:100D10006861766520746865206E6574776F726BA4
:100D200020286E65745F61737365727420616374EB
:100D30006976652900004E6574776F726B20726565
:100D40006C656173656400004E6F77206174207478
:100D5000686520657865637574655F6E65745F634B
:100D60006F6D6D616E642073746570006E65745F85
:100D70007061636B65745F6C656E3D3D00002020A3
:100D8000636D645F64656C696D3D3D002020636D3B
:100D9000645F64656C696D3D3D3D0000636D645F3B
:100DA00064656C696D20203D0000636D645F636F56
:100DB0006D6D616E643D0000636D645F61726720FC
:100DC0002020203D00004F504D4F444500004F4E25
:100DD00044454C41593100004F4E44454C41593235
:100DE00000004F4E44454C41593300004F4E44459E
:100DF0004C41593400004F4E44454C415935000098
:100E00004F464644454C415931004F464644454CB7
:100E1000415932004F464644454C415933004F46F4
:100E20004644454C415934004F464644454C41598F
:100E30003500454E41424C45000044495341424C27
:100E400045004E4F524D414C4F4E00004F6E2073A7
:100E5000657175656E6365203D206E6F726D616CA6
:100E60000000524556455253454F4E004F6E207379
:100E7000657175656E6365203D2072657665727378
:100E800065004E4F524D414C4F4646004F6666201E
:100E900073657175656E6365203D206E6F726D615F
:100EA0006C00524556455253454F464600004F662A
:100EB000662073657175656E6365203D2072657689
:100EC0006572736500004F55543031004F555430F2
:100ED00032004F55543033004F55543034004F5585
:100EE00054303500494E3100494E3200494E3300EE
:100EF00050554C534500435700004B4559004B4556
:100F00005945520057504D004556454E543100004A
:100F10004556454E543200004556454E5433000068
:100F20004556454E543400004556454E5435000054
:100F30004556454E543600004556454E5437000040
:100F4000574D0000574D4C494D4954004144314DD7
:100F5000494E00004144324D494E00004144334D5A
:100F6000494E00004144344D494E00004144314D4A
:100F7000415800004144324D415800004144334D36
:100F8000415800004144344D415800004144414C17
:100F900041524D00414443414C31000041444341E2
:100FA0004C320000414443414C3300004144434132
:100FB0004C340000534554524556000053455442AA
:100FC00055494C4400004E4554004C4F43414C00A1
:100FD00048454C5000004C4F414400005341564599
:100FE000000053544154555300005354415445009C
:100FF000555044415445000044454255474F4E002A
:101000004465627567206D6F6465204F4E004445EE
:101010004255474F464600004465627567206D6F34
:101020006465204F46460000535244454255474FA1
:101030004E005368696674207265676973746572DF
:10104000206465627567206D6F6465204F4E0000F7
:10105000535244454255474F46460000536869661F
:101060007420726567697374657220646562756760
:10107000206D6F6465204F4646004E4554444542FE
:1010800055474F4E00004E6574776F726B20646554
:10109000627567206D6F6465204F4E004E45544465
:1010A000454255474F4646004E6574776F726B2038
:1010B0006465627567206D6F6465204F4646000069
:1010C00050494E470000524F4C4C43414C4C00009D
:1010D000464F5243454641494C0045594543414ED0
:1010E00044590000455945004D5347444952454332
:1010F0005400536574206D657373616765206D6F6F
:10110000646520746F206469726563742E004D53AA
:10111000474E45540000536574206D6573736167D5
:1011200065206D6F646520746F206E6574776F72D3
:101130006B207061636B6574206D6F64652E0000B9
:101140004543484F00005354415445545249474782
:10115000455200005245534554005245424F4F54AA
:1011600000004745544144445200534554414444CF
:1011700052005241440053494C454E5400004D4FDB
:1011800044450000424F4F5400002050494E473A1A
:1011900020002C2046726F6D3A2000002C20416404
:1011A00064726573733A20005354415445313A00D8
:1011B0005354415445313A005354415445313A0057
:1011C0005354415445323A005354415445333A0044
:1011D0005354415445343A005354415445353A0030
:1011E0005354415445313A005354415445323A0026
:1011F0005354415445333A005354415445343A0012
:101200005354415445353A0055504441544500002B
:101210004F4B000053595354454D204641494C2CE7
:101220002066726F6D3A20002E202053687574740A
:10123000696E6720646F776E2E005365742050438B
:1012400020757064617465207472696767657220C7
:10125000746F2000435720444F4E45004F4E00000E
:101260004B65796572206D6F6465204F4E004B654C
:10127000796572206D6F6465204F464600005365A6
:101280007420435720737065656420746F200000DC
:1012900053656E642043573A20002D2D2D2D2D20AF
:1012A000412F4420434F4E564552544552205641FB
:1012B0004C554553202D2D2D2D2D2D2D2D2D000040
:1012C000416E616C6F6720696E2031203D20000007
:1012D00076202046776420202800416E616C6F677D
:1012E00020696E2032203D20000076202052656665
:1012F00020202800416E616C6F6720696E203320CA
:101300003D20000076202020202020202800416E53
:10131000616C6F6720696E2034203D2000007620CC
:1013200020202020202028002D2D2D2D2D2D2D2D6D
:101330002D2D2D2D2D2D2D2D2D2D2D2D2D2D2D2DDD
:101340002D2D2D2D2D2D2D2D2D2D2D2D00004F4EE4
:101350000000416E616C6F6720696E70757420616A
:101360006C61726D206D6F6465204F4E00004F46BA
:101370004600416E616C6F6720696E707574206104
:101380006C61726D206D6F6465204F464600536539
:101390007420412F442031206D696E696D756D2078
:1013A000746F200053657420412F442032206D69F2
:1013B0006E696D756D20746F200053657420412F28
:1013C000442033206D696E696D756D20746F200047
:1013D00053657420412F442034206D696E696D750A
:1013E0006D20746F200053657420412F44203120FC
:1013F0006D6178696D756D20746F20005365742080
:10140000412F442032206D6178696D756D20746FB5
:10141000200053657420412F442033206D6178698A
:101420006D756D20746F200053657420412F44202A
:1014300034206D6178696D756D20746F200053657F
:101440007420412F4420696E7075742031206361CF
:101450006C6962726174696F6E2076616C7565206B
:10146000746F200053657420412F4420696E70759D
:101470007420322063616C6962726174696F6E20DE
:1014800076616C756520746F200053657420412F60
:101490004420696E70757420332063616C696272D8
:1014A0006174696F6E2076616C756520746F2000C1
:1014B00053657420412F4420696E70757420342068
:1014C00063616C6962726174696F6E2076616C75BC
:1014D0006520746F2000212121204C6F7720766FCA
:1014E0006C7461676520616C61726D206F6E20693C
:1014F0006E7075742023302E20204D696E203D20A3
:101500000000762E202041637475616C203D200020
:10151000212121204C6F7720766F6C7461676520E4
:10152000616C61726D206F6E20696E70757420231E
:10153000312E20204D696E203D200000762E202087
:1015400041637475616C203D2000212121204C6F86
:101550007720766F6C7461676520616C61726D20B5
:101560006F6E20696E7075742023322E20204D69B5
:101570006E203D200000762E202041637475616C42
:10158000203D2000212121204C6F7720766F6C7444
:1015900061676520616C61726D206F6E20696E708D
:1015A00075742023332E20204D696E203D200000CD
:1015B000762E202041637475616C203D200021212E
:1015C00021204F76657220766F6C746167652061AB
:1015D0006C61726D206F6E20696E7075742023309F
:1015E0002E20204D6178203D2000762E2020416362
:1015F0007475616C203D2000212121204F76657299
:1016000020766F6C7461676520616C61726D206F0C
:101610006E20696E7075742023312E20204D617804
:10162000203D2000762E202041637475616C203DA2
:101630002000212121204F76657220766F6C746125
:10164000676520616C61726D206F6E20696E7075C8
:10165000742023322E20204D6178203D2000762EEC
:10166000202041637475616C203D200021212120E0
:101670004F76657220766F6C7461676520616C616E
:10168000726D206F6E20696E7075742023332E206A
:10169000204D6178203D2000762E20204163747516
:1016A000616C203D20004F46460057617474206DE8
:1016B000657465722070726F74656374696F6E20F3
:1016C00064697361626C656400004F4E00004261A2
:1016D0007369632077617474206D6574657220701E
:1016E000726F74656374696F6E20656E61626C659C
:1016F0006400435553544F4D0000456E61626C6564
:10170000207573657220646566696E656420776113
:101710007474206D657465722070726F7465637483
:10172000696F6E2072616E6765004B657920696E26
:1017300070757420676F657320696E616374697674
:1017400065004B657920696E70757420676F6573ED
:10175000206163746976650053494C454E5400001E
:10176000564552424F534500426F6F7420696E20B8
:10177000766572626F7365206D6F6465000042521A
:1017800049454600426F6F7420696E206272696538
:1017900066206D6F646500004F4E000053696C65F4
:1017A0006E74206D6F6465204F4646004C4F434178
:1017B0004C004E4554574F524B0043616C6C2073A4
:1017C00069676E2073657420746F20005365742000
:1017D0006669726D776172652072657620746F201C
:1017E0000000536574206669726D776172652062CE
:1017F00075696C6420746F2000004E6574776F7299
:101800006B20616464726573732073657420746FF8
:101810002000536574206D79206E6574776F726B4C
:10182000206164647265737320746F2000005365D7
:1018300074205478204F4E2064656C6179203120EB
:10184000746F2000536574205478204F4E206465D7
:101850006C6179203220746F2000536574205478B5
:10186000204F4E2064656C6179203320746F200016
:10187000536574205478204F4E2064656C61792044
:101880003420746F2000536574205478204F4E200C
:1018900064656C6179203520746F20005365742075
:1018A00052782064656C6179203120746F200000CB
:1018B0005365742052782064656C617920322074FD
:1018C0006F2000005365742052782064656C617944
:1018D000203320746F2000005365742052782064F8
:1018E000656C6179203420746F200000536574208A
:1018F00052782064656C6179203520746F20000077
:101900004F7574707574200020656E61626C65643B
:1019100000004F75747075742000206469736162F3
:101920006C6564004F4E00004F4646005475726E61
:10193000206F75747075742031204F4E00005475FF
:10194000726E206F75747075742031204F4646009A
:101950004F4E00004F4646005475726E206F7574EE
:101960007075742032204F4E00005475726E206FD7
:1019700075747075742032204F4646004F4E00003B
:101980004F4646005475726E206F757470757420E2
:1019900033204F4E00005475726E206F7574707551
:1019A000742033204F4646004F4E00004F464600FD
:1019B0005475726E206F75747075742034204F4E9C
:1019C00000005475726E206F757470757420342029
:1019D0004F4646004F4E00004F4646005475726E0B
:1019E000206F75747075742035204F4E000054754B
:1019F000726E206F75747075742035204F464600E6
:101A00004F4E00004F4646005475726E20696E704E
:101A100075742031204F4E005475726E20696E70BF
:101A200075742031204F464600004F4E00004F464F
:101A300046005475726E20696E7075742032204FA6
:101A40004E005475726E20696E7075742032204F8E
:101A5000464600004F4E00004F4646005475726ED9
:101A600020696E7075742033204F4E005475726E6D
:101A700020696E7075742033204F46460000526511
:101A800073657420616C6C20706172616D65746542
:101A9000727320746F2064656661756C7420766162
:101AA0006C7565732E00436F6E666967757261743D
:101AB000696F6E20736176656420746F20666C6157
:101AC0007368206D656D6F72792E0000436F6E66CE
:101AD000696775726174696F6E206C6F61646564AB
:101AE0002066726F6D20666C617368206D656D6F26
:101AF00072792E00535253205452205365717565EC
:101B00006E63657200002C2028416464723A2000E4
:101B10002D2D2D20545220537175656E63657220F2
:101B2000436F6D6D616E6473202D2D2D2D2D2D2D28
:101B30002D2D2D2D2D2D2D2D2D2D2D2D2D2D2D2DD5
:101B40002D2D2D2D2D2D2D2D2D2D2D2D2D2D2D2DC5
:101B50002D2D2D2D2D2D2D2D2D2D2D2D2D2D2D2DB5
:101B60002D2D00004F4E44454C4159306E207820B9
:101B7000206D732E2044656C617920782028312DEA
:101B80003530303029206D732E206265666F7265A6
:101B9000207475726E696E67206F6E206F75747039
:101BA000757420236E2C20207768657265206E2066
:101BB0003D20312D35004F464644454C4159306E4D
:101BC0002078206D732E2044656C61792078202860
:101BD000312D3530303029206D732E206265666FCF
:101BE0007265207475726E696E67206F6666206F0D
:101BF000757470757420236E2C207768657265206B
:101C00006E203D20312D35004E4F524D414C4F4EF0
:101C10002020202020202020205475726E206F6EFE
:101C20002020696E206E6F726D616C20207365716B
:101C300075656E63652C20312C20322C20332C20CE
:101C4000342C203520202844656661756C74290089
:101C50004E4F524D414C4F46462020202020202000
:101C6000205475726E206F666620696E206E6F72EA
:101C70006D616C202073657175656E63652C203510
:101C80002C20342C20332C20322C203120202844AE
:101C9000656661756C742900524556455253454F2F
:101CA0004E20202020202020205475726E206F6E40
:101CB0002020696E20726576657273652073657188
:101CC00075656E63652C20352C20342C20332C2038
:101CD000322C20310000524556455253454F46465E
:101CE000202020202020205475726E206F666620F0
:101CF000696E2072657665727365207365717565AE
:101D00006E63652C20312C20322C20332C20342C77
:101D100020350000454E41424C45207820202020AF
:101D20002020202020456E61626C6573206F7574E1
:101D300070757420782028312D352900444953418D
:101D4000424C452078202020202020202044697308
:101D500061626C6573206F757470757420782028CB
:101D6000312D352900002D2D2D2041646D696E2007
:101D7000436F6D6D616E6473202D2D2D2D2D2D2DD6
:101D80002D2D2D2D2D2D2D2D2D2D2D2D2D2D2D2D83
:101D90002D2D2D2D2D2D2D2D2D2D2D2D2D2D2D2D73
:101DA0002D2D2D2D2D2D2D2D2D2D2D2D2D2D2D2D63
:101DB0002D2D2D2D2D2D2D2D2D0048454C50202025
:101DC0002020202020202020202020446973706CB7
:101DD000617920746869732068656C7020696E662B
:101DE0006F726D6174696F6E0000535441545553A6
:101DF0002020202020202020202020446973706C87
:101E00006179207468652063757272656E742063F1
:101E10006F6E66696775726174696F6E00004C4F12
:101E20004144202020202020202020202020204C41
:101E30006F616420636F6E66696775726174696F44
:101E40006E2066726F6D20666C617368206D656DC3
:101E50006F727900534156452020202020202020F9
:101E600020202020205361766520636F6E666967AD
:101E700075726174696F6E20746F20666C6173682F
:101E8000206D656D6F7279005245534554202020B6
:101E90002020202020202020205265736574206F90
:101EA0007065726174696E6720706172616D6574CE
:101EB00065727320746F207374616E646172642044
:101EC00064656661756C742076616C75657300007D
:101ED0005245424F4F5420202020202020202020F7
:101EE000205265626F6F7420746865207379737413
:101EF000656D0000424F4F542053494C454E5420CD
:101F000020202020205475726E73206F6666206238
:101F10006F6F74206D65737361676500424F4F5436
:101F200020564552424F53452020202020547572A0
:101F30006E73206F6E20626F6F74206D65737361B6
:101F40006765000053544154455452494747455230
:101F50002078787820557064617465732050432030
:101F600070726F6772616D20646973706C61792043
:101F700069662064656C6179206973203E207878F9
:101F800078202864656661756C74203D2032353098
:101F9000206D732900002D2D2D20412F4420436FEB
:101FA0006E766572746572202D20416E616C6F676C
:101FB00020496E7075742043616C69627261746946
:101FC0006F6E2D2D2D2D2D2D2D2D2D2D2D2D2D2DBE
:101FD0002D2D2D2D2D2D2D2D2D2D2D2D2D2D2D2D31
:101FE0002D2D2D2D2D2D2D2D2D00414443414C6E99
:101FF0002078787820202020202020416473206FD2
:1020000072207375627472616374732074686520E2
:102010006F6666736574207878782028696E206D05
:10202000696C69766F6C74732920746F20746865AD
:1020300020412F4420636F6E76657274657220278D
:102040006E27202028312D34290041446E4D494E01
:102050002078787820202020202020536574732059
:102060006C6F77207472696767657220616C61724A
:102070006D20766F6C7461676520746F2078787856
:1020800020766F6C74732028696E20766F6C747381
:10209000290041446E4D4158207878782020202036
:1020A0002020205365747320686967682074726902
:1020B0006767657220616C61726D20766F6C746108
:1020C000676520746F2078787820766F6C74732041
:1020D00028696E20766F6C74732900005241442089
:1020E0002020202020202020202020202052656138
:1020F0006420616E616C6F6720696E707574207604
:102100006F6C74616765206E6F7700002D2D2D2038
:10211000435720436F6D6D616E6473202D2D2D2DFF
:102120002D2D2D2D2D2D2D2D2D2D2D2D2D2D2D2DDF
:102130002D2D2D2D2D2D2D2D2D2D2D2D2D2D2D2DCF
:102140002D2D2D2D2D2D2D2D2D2D2D2D2D2D2D2DBF
:102150002D2D2D2D2D2D2D2D2D2D2D2D2D2D2D00DC
:102160004B45594552204F4E202020202020202032
:10217000205475726E206F6E206B65796572206DCC
:102180006F64652E20204F7574707574203520772C
:10219000696C6C2073656E64204357207573696E9B
:1021A000672074686520435720636F6D6D616E64AE
:1021B00000004B45594552204F4646202020202004
:1021C0002020205475726E206F6666206B657965DD
:1021D00072206D6F64652E20204F757470757420A9
:1021E000352077696C6C206F706572617465206949
:1021F0006E206E6F726D616C2073657175656E63B4
:102200006572206D6F646500435720787878787820
:1022100020202020202020202053656E642074651B
:10222000787420787878787820696E204357207504
:1022300073696E67206F7574707574203520696ED0
:10224000206B65796572206D6F64650057504D2075
:102250007878202020202020202020202053657402
:1022600020435720737065656420696E206170702B
:10227000726F78696D61746520776F726473207016
:102280006572206D696E7574652028312D39392984
:1022900000002D2D2D204E6574776F726B20436FDB
:1022A0006D6D616E6473202D2D2D2D2D2D2D2D2DF9
:1022B0002D2D2D2D2D2D2D2D2D2D2D2D2D2D2D2D4E
:1022C0002D2D2D2D2D2D2D2D2D2D2D2D2D2D2D2D3E
:1022D0002D2D2D2D2D2D2D2D2D2D2D2D2D2D2D2D2E
:1022E0002D2D2D2D2D0053455441444452207878F6
:1022F00020202020202020576865726520787820D3
:1023000069732074686520626F6172642773206E40
:102310006574776F726B20616464726573732028D3
:102320006265747765656E203120616E6420313599
:102330002900474554414444522020202020202099
:10234000202020476574207468652076616C75656F
:10235000206F662074686520626F61726427732045
:102360006E6574776F726B2061646472657373005D
:1023700053494C454E54204F4E20202020202020F1
:1023800020446F206E6F742073656E64206D6573DA
:10239000736167657320746F2073657269616C2067
:1023A000706F7274207768656E2073746174652035
:1023B0006368616E6765730053494C454E54204F06
:1023C00046462020202020202053656E64206D6525
:1023D00073736167657320746F2073657269616CD4
:1023E00020706F7274207768656E207374617465F5
:1023F000206368616E67657300002D2D2D204D618F
:102400006E75616C204F757470757420436F6D6DBF
:10241000616E6473202D2D2D2D2D2D2D2D2D2D2D07
:102420002D2D2D2D2D2D2D2D2D2D2D2D2D2D2D2DDC
:102430002D2D2D2D2D2D2D2D2D2D2D2D2D2D2D2DCC
:102440002D2D2D2D2D2D2D2D2D2D2D2D2D004F559F
:1024500054306E204F4E2020202020202020204D60
:10246000616E75616C6C79207475726E204F4E20B0
:10247000206F7574707574206E2028312D352900F9
:102480004F5554306E204F464620202020202020DB
:10249000204D616E75616C6C79207475726E204F81
:1024A0004646206F7574707574206E2028312D3566
:1024B00029002D2D2D2D2D2D2D2D2D2D2D2D2D2D7D
:1024C0002D2D2D2D2D2D2D2D2D2D2D2D2D2D2D2D3C
:1024D0002D2D2D2D2D2D2D2D2D2D2D2D2D2D2D2D2C
:1024E0002D2D2D2D2D2D2D2D2D2D2D2D2D2D2D2D1C
:1024F0002D2D2D2D2D2D2D2D2D2D2D2D2D2D2D2D0C
:102500002D2D2D2D2D0020202020202020202020AA
:1025100020202020202020466F72206D6F726520C1
:10252000696E666F726D6174696F6E20676F20747B
:102530006F207777772E7369657272617261646953
:102540006F2E6E6574002D2D2D2D2D2D2D2D2D2DE5
:102550002D2D2D2D2D2D2D2D2D2D2D2D2D2D2D2DAB
:102560002D2D2D2D2D2D2D2D2D2D2D2D2D2D2D2D9B
:102570002D2D2D2D2D2D2D2D2D2D2D2D2D2D2D2D8B
:102580002D2D2D2D2D2D2D2D2D2D2D2D2D2D2D2D7B
:102590002D2D2D2D2D2D2D2D2D003D3D3D3D3D5B1A
:1025A0002043555252454E5420434F4E46494755BD
:1025B000524154494F4E205D3D3D3D3D3D3D3D3DE9
:1025C0003D00436F6E66696720636F646520203A43
:1025D0002000426F61726420747970652020203A77
:1025E000200046572076657273696F6E2020203A6E
:1025F00020004657206275696C6420202020203A14
:1026000020004D7920616464726573732020203A44
:1026100020004F4E202064656C6179203120203AE3
:1026200020004F4E202064656C6179203220203AD2
:1026300020004F4E202064656C6179203320203AC1
:1026400020004F4E202064656C6179203420203AB0
:1026500020004F4E202064656C6179203520203A9F
:1026600020004F46462064656C6179203120203A75
:1026700020004F46462064656C6179203220203A64
:1026800020004F46462064656C6179203320203A53
:1026900020004F46462064656C6179203420203A42
:1026A00020004F46462064656C6179203520203A31
:1026B00020003A20456E61626C6564003A2044490E
:1026C0005341424C454400004F757470757420317D
:1026D0002020202020003A20456E61626C65640055
:1026E0003A2044495341424C454400004F757470B0
:1026F000757420322020202020003A20456E61622F
:102700006C6564003A2044495341424C4544000002
:102710004F757470757420332020202020003A20DB
:10272000456E61626C6564003A2044495341424CF5
:10273000454400004F7574707574203420202020AB
:1027400020003A20456E61626C6564003A2044497D
:102750005341424C454400004F75747075742035E8
:102760002020202020004F4E2073657175656E6318
:102770006520203A204E6F726D616C004F4E2073C1
:10278000657175656E636520203A205265766572C5
:10279000736564004F46462073657175656E6365A9
:1027A000203A204E6F726D616C004F464620736573
:1027B0007175656E6365203A205265766572736542
:1027C0006400435720737065656420202020203A00
:1027D000200057617474206D6574657220636865AC
:1027E000636B696E67204F46460053696D706C6578
:1027F0002077617474206D65746572206368656309
:102800006B696E6720656E61626C6564000057617C
:102810007474206D65746572206C696D69742073C1
:10282000657420746F200000414420616C61726DFA
:10283000206D6F64653A204F666600004144206158
:102840006C61726D206D6F64653A204F4E00416E71
:10285000616C6F672031206D696E203A2000202066
:10286000202020202020206D6178203A2000202088
:102870002020202020202063616C203A2000416E1F
:10288000616C6F672032206D696E203A2000202035
:10289000202020202020206D6178203A2000202058
:1028A0002020202020202063616C203A2000416EEF
:1028B000616C6F672033206D696E203A2000202004
:1028C000202020202020206D6178203A2000202028
:1028D0002020202020202063616C203A2000416EBF
:1028E000616C6F672034206D696E203A20002020D3
:1028F000202020202020206D6178203A20002020F8
:102900002020202020202063616C203A2000436F8B
:102910006D6D206D6F6465202020203A204C6F6320
:10292000616C0000436F6D6D206D6F646520202029
:10293000203A204E6574776F726B0000F86A400E83
:10294000386E006A030EAF6E200EAC6E900EAB6E4A
:102950002EEE81F094988298949A829A9390819026
:102960009392819293948194110E05012F6FC70E5B
:102970002E6F510E2D6F810E2C6F0101D99DD98FB5
:10298000040E196EB00E186E1D6A91C51CF09CECF9
:1029900002F005018F6F19C090F5030E8E6F520E75
:1029A0008D6F05EEE4F0540EEE6E520EEE6E310EAB
:1029B000EE6EEF6A000114EF15F09EAA23D0060E0A
:1029C000AB141DE1E2CF3DF0E1CF3CF03E2AFF0E1B
:1029D0003E5C01E33E6A1DEE82F03E50E126000EB1
:1029E000E222AECFE7FF0D0EE75C02E1010E426E80
:1029F0003EC018F43DC0E2FF3CC0E1FF1100AB98BF
:102A0000AB8800D011003E6A3F6A9D8AC00EF26E0C
:102A100012009D9A0DEE82F0FF0EEE6AE82EFDD7B1
:102A20003E6A3F6A9D8A1200400EAF6E900EAB6EFA
:102A3000200EAC6E0B0EC16EF19E320E24EC02F035
:102A40008298829A819081928194939481949392B6
:102A5000819293908190949A829A9498829801019D
:102A6000D99BD9BF8282D9AF829205012B910101F6
:102A7000CC6BD46BDB6BDA6B01EEDCF04F0EEE6EE1
:102A80004B0EEE6EEF6A020EE16F01EE1CF0EE6A85
:102A900001EEE2F0EE6A0401A16B640EA06FA36B7D
:102AA000A26B04EE1AF0300EEE6EEE6EEF6A0601C7
:102AB0001189118B119D0401A46B04EEA5F0EE6A3F
:102AC0000501286B276BEE89EE8BEE8DEE8F0601EC
:102AD000118111930501786BCD0E7C6FCC0E7B6F4D
:102AE0004C0E7A6F7C0E796F0601119511970101DA
:102AF000686B6A6B0501266B4B6B4A6B496B486BC5
:102B00004F6B4E6B4D6B4C6B536B526B516B506BF1
:102B1000576B566B556B546B01016B6B05015B6B0F
:102B20005A6B596B586B5F6B5E6B5D6B5C6B636B69
:102B3000626B616B606B676B666B656B646B6B6B19
:102B40006A6B700E696F830E686F6F6B6E6B700EC1
:102B50006D6F830E6C6F736B726B700E716F830E83
:102B6000706F776B766B700E756F830E746F0101EB
:102B70006C6B49DF0001E9EC17F00101D991D993A1
:102B8000D995010E0501EB6F010EDF6FE16B050EAC
:102B9000E06FE36B070EE26F010EED6F5B6B5A6B3C
:102BA000596B586B6B6B6A6B200E696F810E686F87
:102BB0005F6B5E6B5D6B5C6B6F6B6E6B200E6D6F36
:102BC000810E6C6F636B626B616B606B736B726BAE
:102BD000200E716F810E706F676B666B656B646B37
:102BE000776B766B200E756F810E746FEE972A6B84
:102BF000640E296FEB29EC6F0001B9EC2AF082B664
:102C000003EF16F0F9D794908280000EF5EC01F0F6
:102C10000501DF6FDF290001D8A43AEF16F00401A7
:102C2000A4530001D8A43AEF16F004EEA5F00A0E62
:102C3000F76E420EF66ED9EC02F0EF6AE4EC1DF08E
:102C400004EEA5F00A0EF76E6A0EF66ED9EC02F0ED
:102C5000EF6AE4EC1DF0B5EC45F064EC46F004EEF0
:102C6000A5F00A0EF76E820EF66ED9EC02F0EF6A4E
:102C7000E4EC1DF0D8EC49F00AEC39F001EE6DF00F
:102C8000020E016E0501ED51CCEC00F0EF6A010E71
:102C90000401A453D8A4000E356E010E01016B533C
:102CA000D8A4000E35140001D8B4CCEF16F004EE11
:102CB000A5F00A0EF76EAA0EF66ED9EC02F0EF6AD6
:102CC000E4EC1DF004EEA5F00A0EF76ED20EF66EDF
:102CD000D9EC02F0EF6AE4EC1DF004EEA5F00A0E68
:102CE000F76EF40EF66ED9EC02F0020E016E086A71
:102CF000E1C521F0E0C520F0CFEC00F00B0EF76E3F
:102D0000060EF66ED9EC02F0020E016E086AE3C5FB
:102D100021F0E2C520F0CFEC00F0EF6AE4EC1DF00A
:102D200004EEA5F00B0EF76E100EF66ED9EC02F065
:102D3000020E016E0501ED51CCEC00F0EF6A04EEDD
:102D4000A5F00B0EF76E220EF66ED9EC02F0EF6ACC
:102D50000001E4EC1DF004EEA5F00B0EF76E440E3E
:102D6000F66ED9EC02F0EF6AE4EC1DF004EEA5F08B
:102D70000B0EF76E6C0EF66ED9EC02F0EF6AE4EC17
:102D80001DF004EEA5F00B0EF76E7C0EF66ED9EC7E
:102D900002F0EF6ACAEC1DF0320E24EC02F09490BF
:102DA00082900B0EF76E880EF66E01EEDCF001ECF1
:102DB00003F0D8A4DEEF16F01AEC2BF0D89606013B
:102DC00011ADD8860001D8B6E8EF16F01DEF17F068
:102DD00001EEA0F0020E016EE86A80BA010ECCECA2
:102DE00000F0EF6A01EEA0F084EC00F0808AE8A029
:102DF000809A01EEB5F0020E016EE86A81B6010E0E
:102E0000CCEC00F0EF6A01EEB5F084EC00F08186C6
:102E1000E8A081962CEC30F0010E01016C5D000100
:102E2000D8A415EF17F0EEEC35F00501785300014A
:102E3000D8B41DEF17F095EC38F00601119D010E86
:102E40000101E15D0001D8A428EF17F098EF17F019
:102E5000020E0101E15D0001D8A431EF17F033EF5C
:102E600017F0A9EF17F081A838EF17F025EF40F021
:102E7000010E0101CC6FE86A80BA010E356EE86A76
:102E800081B6010E35100001D8B44CEF17F00101E6
:102E9000CC6B00014FEF17F0010E0101CC6F000168
:102EA000010E0101CC5D010ED8A4000E356E010E9D
:102EB00005012BBDE86A35140001D8B462EF17F0A4
:102EC00016EF40F0010E0101CC5D010ED8A4000EFA
:102ED000356EE86A05012BBD010E35140001D8B42A
:102EE00074EF17F089EF3AF0010E0101CC53D8A42A
:102EF000000E356E010E05012BBDE86A3514000188
:102F0000D8B485EF17F057EF3DF0010E0101CC5317
:102F1000D8A4000E356EE86A05012BBD010E3514EC
:102F20000001D8B496EF17F01BEF40F0A9EF17F0AF
:102F300080AA9DEF17F01BEC39F081A6A2EF17F0E5
:102F400054EC39F081A8A7EF17F08DEC39F0A9EF18
:102F500017F00501274B282B2751295D28512A59A5
:102F60000001D8B0D2EF17F00501286B276BD89677
:102F70002BB1D8860001D8B6C5EF17F005012B811B
:102F8000949282920001D2EF17F0D89605012BA1FE
:102F9000D8860001D8B6D1EF17F005012B91949295
:102FA000828200010401A251A05DA351A159000138
:102FB000D8B0E0EF17F0E9EC17F00401A36BA26BB7
:102FC0000001010E425CD8A4E8EF17F0EDEC17F019
:102FD000E8D6426A09EC15F01200D8960101D9A58D
:102FE000D8860001D8B601EF18F00B0EF76E8E0EE2
:102FF000F66ED7EC01F00D0EDFEC01F00A0EDFECFF
:1030000001F001EEE2F0820EEE6AE82EFDD7D896CE
:103010000101D9A5D8860001D8B625EF18F00B0E0E
:10302000F76EA00EF66ED7EC01F001EEE2F0EE5076
:1030300003E0DFEC01F0FBD73E0EDFEC01F00D0EFC
:10304000DFEC01F00A0EDFEC01F03E040401186F22
:1030500000013EAE2EEF18F00401186B0001D89667
:103060000101D9A5D8860001D8B649EF18F00B0E9A
:10307000F76EBE0EF66ED7EC01F0040E016E040181
:103080001851CCEC00F00D0EDFEC01F00A0EDFEC75
:1030900001F00001040118530001D8A453EF18F007
:1030A000010E0401186F0001040118050B6E0101E7
:1030B000CC6B00010101CC510B5C0001D8A099EF51
:1030C00018F0D8960101CCAFD8860001D8B66BEFC6
:1030D00018F00101CC6B00010101CC290DEE82F04A
:1030E000E926000EEA22EFCF0FF001EEE2F0CC511C
:1030F000E926000EEA220FC0EFFFD896D9A5D886A0
:103100000001D8B693EF18F0040E016E01EEE2F064
:103110000101CC51E926000EEA22EF50CCEC00F080
:10312000200EDFEC01F000010101CC2B0001D8A43E
:10313000C0D79CEC18F0120001EEE2F011EEE2F0C4
:10314000F5EC02F0D8960101D9A5D8860001D8B6D1
:10315000BDEF18F00B0EF76ED00EF66ED7EC01F047
:1031600001EEE2F0EE5003E0DFEC01F0FBD70D0ED4
:10317000DFEC01F00A0EDFEC01F002EE64F011EE7C
:10318000E2F0010EF36E010EE1EC02F0EF6AD89668
:103190000101D9A5D8860001D8B6E2EF18F00B0ED0
:1031A000F76EDA0EF66ED7EC01F002EE64F0EE5038
:1031B00003E0DFEC01F0FBD70D0EDFEC01F00A0EAF
:1031C000DFEC01F002EE66F011EEE2F0020EF36EBB
:1031D000010EE1EC02F0EF6AD8960101D9A5D8867C
:1031E0000001D8B607EF19F00B0EF76EE40EF66E7D
:1031F000D7EC01F002EE66F0EE5003E0DFEC01F0F8
:10320000FBD70D0EDFEC01F00A0EDFEC01F002EE51
:1032100069F011EEE2F0030EF36E020EE1EC02F043
:10322000EF6AD8960101D9A5D8860001D8B62CEF4F
:1032300019F00B0EF76EEE0EF66ED7EC01F002EE03
:1032400069F0EE5003E0DFEC01F0FBD70D0EDFEC90
:1032500001F00A0EDFEC01F002EE6DF011EEE2F08B
:10326000050EF36E020EE1EC02F0EF6AD896010152
:10327000D9A5D8860001D8B651EF19F00B0EF76E1C
:10328000F80EF66ED7EC01F002EE6DF0EE5003E0B2
:10329000DFEC01F0FBD70D0EDFEC01F00A0EDFECE6
:1032A00001F002EE71F011EEE2F0070EF36E030E84
:1032B000E1EC02F0EF6AD8960101D9A5D8860001A9
:1032C000D8B676EF19F00C0EF76E000EF66ED7EC4E
:1032D00001F002EE71F0EE5003E0DFEC01F0FBD7FD
:1032E0000D0EDFEC01F00A0EDFEC01F002EE76F0DD
:1032F00011EEE2F00A0EF36E090E0401185DE1EC26
:1033000002F0EF6AD8960101D9A5D8860001D8B697
:10331000A0EF19F00C0EF76E0A0EF66ED7EC01F066
:1033200002EE76F0EE5003E0DFEC01F0FBD73E0E4C
:10333000DFEC01F00D0EDFEC01F00A0EDFEC01F026
:1033400001EEE2F0E86AEE5202E0E83EFCD704014A
:10335000186FD8960101D9A5D8860001D8B6C3EF59
:1033600019F00C0EF76E180EF66ED7EC01F0040E85
:10337000016E04011851CCEC00F00D0EDFEC01F0F1
:103380000A0EDFEC01F0000102EE76F0E86AEE5280
:1033900002E0E83EFCD70401196FD8960101D9A5D7
:1033A000D8860001D8B6E7EF19F00C0EF76E280E9C
:1033B000F66ED7EC01F0040E016E04011951CCEC4D
:1033C00000F00D0EDFEC01F00A0EDFEC01F0000161
:1033D00004EE1AF012EE69F0030EE75204E0E6CFB5
:1033E000EEFFE82EFAD7EF6A300E0201665D0001AB
:1033F000D8A4FDEF19F0A1EF1BF02F0E0201665DBE
:103400000001D8A406EF1AF00101D98B00012F0E9C
:103410000201665D0001D8A413EF1AF004EE1AF061
:10342000300EEE6EEF6A2F0E0201665D0001D8A429
:103430001CEF1AF06EEC1FF02F0E0201665D00010A
:10344000D8A428EF1AF001016A6B00012BEF1AF0E3
:10345000010E01016A6F00012F0E0201665D00017D
:10346000D8A434EF1AF01200D8960101D9A5D88655
:103470000001D8B648EF1AF00C0EF76E3A0EF66E51
:10348000D7EC01F00D0EDFEC01F00A0EDFEC01F0DD
:10349000D8960101D9A5D8860001D8B662EF1AF0F6
:1034A0000C0EF76E500EF66ED7EC01F0040E016EA6
:1034B0000101D451CCEC00F00D0EDFEC01F00A0E4E
:1034C000DFEC01F000010401176B010E0101CC6F6C
:1034D0000001060E0101CC5D0001D8B0CCEF1AF05E
:1034E00001EEE2F00101CC51E926000EEA22EF5094
:1034F000D46FD4510401171B01EEA0F0020E016E2F
:103500000101CC51CCEC00F0EF6A01EEB5F0020EF7
:10351000016E04011751CCEC00F0EF6AD89601015E
:10352000D9A5D8860001D8B6C6EF1AF001EEA0F0F2
:10353000EE5003E0DFEC01F0FBD7200EDFEC01F0F2
:1035400001EEE2F00101CC51E926000EEA22EF5033
:10355000DFEC01F0200EDFEC01F0630EDFEC01F098
:10356000720EDFEC01F0630EDFEC01F03D0EDFECDC
:1035700001F001EEB5F0EE5003E0DFEC01F0FBD717
:103580000D0EDFEC01F00A0EDFEC01F0000101018D
:10359000CC2B0001D8A49CD7090E0101CC6F0001EF
:1035A0000101CC510401185D0001D8A034EF1BF0DB
:1035B00001EEE2F00101CC51E926000EEA22EF50C3
:1035C0000B6E0B500401171B01EEA0F0020E016EF2
:1035D0000101CC51CCEC00F0EF6A01EEB5F0020E27
:1035E000016E04011751CCEC00F0EF6AD89601018E
:1035F000D9A5D8860001D8B62EEF1BF001EEA0F0B9
:10360000EE5003E0DFEC01F0FBD7200EDFEC01F021
:1036100001EEE2F00101CC51E926000EEA22EF5062
:10362000DFEC01F0200EDFEC01F0630EDFEC01F0C7
:10363000720EDFEC01F0630EDFEC01F03D0EDFEC0B
:1036400001F001EEB5F0EE5003E0DFEC01F0FBD746
:103650000D0EDFEC01F00A0EDFEC01F000010101BC
:10366000CC2B0001D8A49BD7D8960101D9A5D88628
:103670000001D8B65BEF1BF00C0EF76E620EF66E13
:10368000D7EC01F0040E016E04011751CCEC00F0F0
:103690000C0EF76E740EF66ED7EC01F002EE71F0C0
:1036A000EE5003E0DFEC01F0FBD70D0EDFEC01F094
:1036B0000A0EDFEC01F0000102EE71F084EC00F084
:1036C0000B6E21C00CF022C00DF023C00EF00D5087
:1036D0000E100AE10C500D1007E10B5004011719F0
:1036E0000001D8B48DEF1BF0D8960101D9A5D8867A
:1036F0000001D8B688EF1BF00C0EF76E840EF66E44
:10370000D7EC01F00D0EDFEC01F00A0EDFEC01F05A
:10371000E9EC17F01200A1EF1BF0D8960101D9A532
:10372000D8860001D8B6A1EF1BF00C0EF76E9C0EE8
:10373000F66ED7EC01F00D0EDFEC01F00A0EDFECB7
:1037400001F0D8960101D9A5D8860001D8B6BBEF03
:103750001BF00C0EF76EB60EF66ED7EC01F0040EF1
:10376000016E0501ED51CCEC00F00D0EDFEC01F027
:103770000A0EDFEC01F0000102EE6DF084EC00F0C7
:103780000101D46FD76BD4510501ED5D0001D8A4C0
:10379000CDEF1BF0010E0101D76F0001630E010197
:1037A000D45D0001D8A4D8EF1BF0010E0101D76F42
:1037B0000001630E0101D45D0001D8A4E3EF1BF00A
:1037C000020E01016A6F0001010E0101D75D0001C7
:1037D000D8A409EF1CF0D8960101D9A5D88600011C
:1037E000D8B6FFEF1BF00C0EF76EC20EF66ED7ECDC
:1037F00001F00D0EDFEC01F00A0EDFEC01F002EE3D
:1038000076F012EE76F0F5EC02F085EC1FF01DEF8D
:103810001CF0D8960101D9A5D8860001D8B61DEFB5
:103820001CF00C0EF76EDE0EF66ED7EC01F00D0EEE
:10383000DFEC01F00A0EDFEC01F0E9EC17F012000A
:1038400002EECBF011EE31F0360EE75204E0E6CF97
:10385000EEFFE82EFAD7EF6A31EC1CF0D9EC1EF03F
:10386000120003EE0DF0820EEE6AE82EFDD702EE96
:10387000B8F02F0EEE6EEF6A02EEBBF0410EEE6E68
:10388000EF6A02EEBEF0020E016E0501ED51CCECC6
:1038900000F0EF6A02EEBEF0E86AEE5202E0E83EA7
:1038A000FCD70B6E010E0B5C0001D8A468EF1CF076
:1038B00001EEB5F0300EEE6E12EEBEF0030EE752E2
:1038C00004E0E6CFEEFFE82EFAD7EF6A74EF1CF0C3
:1038D00001EEB5F012EEBEF0030EE75204E0E6CFC3
:1038E000EEFFE82EFAD7EF6A02EEBEF011EEB5F069
:1038F000140EE75204E0E6CFEEFFE82EFAD7EF6AA7
:1039000002EEC2F014EE1AF0030EE75204E0E6CF26
:10391000EEFFE82EFAD7EF6A02EEC2F0E86AEE5246
:1039200002E0E83EFCD70101D46FD4530001D8A4D3
:10393000A0EF1CF002EEC2F0300EEE6EEE6EEF6AFB
:10394000010E0101D45D0001D8A4C1EF1CF004EE0A
:10395000A5F0300EEE6E12EEC2F0030EE75204E058
:10396000E6CFEEFFE82EFAD7EF6A02EEC2F014EED1
:10397000A5F0800EE75204E0E6CFEEFFE82EFAD77E
:10398000EF6A020E0101D45D0001D8A4CEEF1CF055
:1039900002EEC2F0EE50FEE1ED52EF6A01EE6DF084
:1039A00012EEB8F0020EE75204E0E6CFEEFFE82E8A
:1039B000FAD712EEBBF0020EE75204E0E6CFEEFFBC
:1039C000E82EFAD712EEBEF0030EE75204E0E6CF7F
:1039D000EEFFE82EFAD712EEC2F0030EE75204E033
:1039E000E6CFEEFFE82EFAD712EECBF0410EE7520B
:1039F00004E0E6CFEEFFE82EFAD7EF6A01EE6DF0B5
:103A0000E86AEE5202E0E83EFCD70101D86FD76BBE
:103A100001EE6DF0E86AEE5202E0E83EFCD70B6E74
:103A2000010ECC6F00010101CC510B5C0001D8A04C
:103A300036EF1DF001EE6DF00101CC51EB50D46F6B
:103A4000D451D71B01EEA0F0020E016ECC51CCEC8C
:103A500000F0EF6A01EEB5F0020E016ED751CCEC2A
:103A600000F0EF6ACC2B0001D8A4DCD702EEC6F040
:103A7000020E016E0101D751CCEC00F0EF6A02EEAC
:103A8000C6F0E86AEE5202E0E83EFCD7D46F010EC1
:103A9000D45D0001D8A45CEF1DF004EEA5F0300E5B
:103AA000EE6EEE6E12EEC6F0040EE75204E0E6CFC4
:103AB000EEFFE82EFAD7EF6A020E0101D45D000195
:103AC000D8A471EF1DF004EEA5F0300EEE6E12EEEC
:103AD000C6F0040EE75204E0E6CFEEFFE82EFAD778
:103AE000EF6A030E0101D45D0001D8A484EF1DF03C
:103AF00004EEA5F012EEC6F0040EE75204E0E6CFA5
:103B0000EEFFE82EFAD7EF6A02EEC6F014EEA5F04B
:103B1000800EE75204E0E6CFEEFFE82EFAD7EF6A18
:103B200003EE0DF012EEB8F0020EE75204E0E6CF1D
:103B3000EEFFE82EFAD712EEBBF0020EE75204E0D9
:103B4000E6CFEEFFE82EFAD712EEBEF0030EE752F4
:103B500004E0E6CFEEFFE82EFAD712EEC2F0030E35
:103B6000E75204E0E6CFEEFFE82EFAD712EEC6F0F9
:103B7000040EE75204E0E6CFEEFFE82EFAD712EE8D
:103B8000CBF0410EE75204E0E6CFEEFFE82EFAD785
:103B9000EF6A1200800E026E100E096E400E296E42
:103BA000540E286E066A056A200E016E810E076E9D
:103BB000040E216EA50E82EC01F00D0E93EC01F0C7
:103BC0000A0E93EC01F0120001016A530001D8A41F
:103BD00032EF1EF00EEC1FF0D8960101D9A5D88661
:103BE0000001D8B607EF1EF00C0EF76EEE0EF66E63
:103BF000D7EC01F004EEA5F0EE5003E0DFEC01F0AD
:103C0000FBD70D0EDFEC01F00A0EDFEC01F0040132
:103C1000A4530001D8A41AEF1EF004EEA5F0EE5054
:103C200003E0DFEC01F0FBD70D0EDFEC01F00A0E34
:103C3000DFEC01F0010E0401A45D0001D8A42EEF19
:103C40001EF004EEA5F0EE5003E0DFEC01F0FBD730
:103C50000D0EDFEC01F00A0EDFEC01F057EC1FF067
:103C6000D8EF1EF0010E01016A5D0001D8A481EFBA
:103C70001EF00EEC1FF0D8960101D9A5D8860001E0
:103C8000D8B656EF1EF00C0EF76EF60EF66ED7ECA9
:103C900001F004EEA5F0EE5003E0DFEC01F0FBD7FD
:103CA0000D0EDFEC01F00A0EDFEC01F00401A4536D
:103CB0000001D8A469EF1EF004EEA5F0EE5003E079
:103CC000DFEC01F0FBD70D0EDFEC01F00A0EDFECAC
:103CD00001F0010E0401A45D0001D8A47DEF1EF0E7
:103CE00004EEA5F0EE5003E0DFEC01F0FBD70D0E83
:103CF000DFEC01F00A0EDFEC01F057EC1FF0D8EF1B
:103D00001EF0020E01016A5D0001D8A4D8EF1EF07A
:103D10000501ED51320DF3CF1CF0F4CF1DF026EC70
:103D200002F000010EEC1FF0D8960101D9A5D8864B
:103D30000001D8B6AFEF1EF00C0EF76EFE0EF66E59
:103D4000D7EC01F004EEA5F0EE5003E0DFEC01F05B
:103D5000FBD70D0EDFEC01F00A0EDFEC01F00401E1
:103D6000A4530001D8A4C2EF1EF004EEA5F0EE505B
:103D700003E0DFEC01F0FBD70D0EDFEC01F00A0EE3
:103D8000DFEC01F0010E0401A45D0001D8A4D6EF20
:103D90001EF004EEA5F0EE5003E0DFEC01F0FBD7DF
:103DA0000D0EDFEC01F00A0EDFEC01F057EC1FF016
:103DB00012000EEC1FF0D8960101D9A5D88600019B
:103DC000D8B6F6EF1EF00D0EF76E060EF66ED7ECB7
:103DD00001F003EE0DF0EE5003E0DFEC01F0FBD755
:103DE0000D0EDFEC01F00A0EDFEC01F0D8960601B3
:103DF00011B7D8860001D8B60BEF1FF003EE0DF017
:103E0000EE5003E0DFEC01F0FBD70D0EDFEC01F02C
:103E10000A0EDFEC01F057EC1FF012000101D76B26
:103E2000000101EEA0F0020E016EE86A82B6010EFA
:103E3000CCEC00F0EF6A01EEA0F084EC00F00101A0
:103E4000D46F010ED45D0001D8A429EF1FF03DEF1F
:103E50001FF00101D72B0501ED510A0DF3CF1CF026
:103E6000F4CF1DF026EC02F0330E0101D75D000106
:103E7000D8A03CEF1FF01200D3D794908280050E9B
:103E800024EC02F0D8960101D9A5D8860001D8B655
:103E900056EF1FF00D0EF76E0E0EF66ED7EC01F01A
:103EA0000D0EDFEC01F00A0EDFEC01F01200949031
:103EB0008290D8960101D9A5D8860001D8B66DEFB9
:103EC0001FF00D0EF76E360EF66ED7EC01F00D0EEC
:103ED000DFEC01F00A0EDFEC01F01200D8960101D0
:103EE000D9ABD8860001D8B684EF1FF002EE76F089
:103EF00011EEE2F0030EF36E000E0401185DE1EC2A
:103F000002F0EF6A0101D99B0001D8960101D9A501
:103F1000D8860001D8B699EF1FF00D0EF76E480E47
:103F2000F66ED7EC01F00D0EDFEC01F00A0EDFECBF
:103F300001F001EEE2F012EE76F0410EE75204E0FD
:103F4000E6CFEEFFE82EFAD7EF6A416A01EEE2F023
:103F5000E86AEE5202E0E83EFCD70401186F010166
:103F6000CC6B00010101CC510401185D0001D8A007
:103F70003DEF20F0D8960101D9A5D8860001D8B62A
:103F8000D4EF1FF00D0EF76E6C0EF66ED7EC01F04D
:103F9000040E016E04011851CCEC00F00D0EDFECA4
:103FA00001F00A0EDFEC01F00001D8960101D9A55D
:103FB000D8860001D8B6FAEF1FF0690EDFEC01F0E9
:103FC0003D0EDFEC01F0DFEC01F0040E016E0101AB
:103FD000CC51CCEC00F00D0EF76E7E0EF66ED7ECE9
:103FE00001F04150CCEC00F00D0EDFEC01F00A0EB8
:103FF000DFEC01F0000101EEE2F00101CC51E92615
:10400000000EEA22EF500B6E200E0B5C0001D8A4CC
:1040100010EF20F00101CC29416E00013DEF20F0AE
:10402000D8960101D9A5D8860001D8B637EF20F07F
:10403000690EDFEC01F03D0EDFEC01F0DFEC01F08A
:10404000DFEC01F0040E016E0101CC51CCEC00F06C
:104050000D0EF76E8C0EF66ED7EC01F04150CCECE5
:1040600000F00D0EDFEC01F00A0EDFEC01F00001B4
:104070000101CC2B0001D8A474D700EE43F011EE5F
:10408000E2F04104E6CFEEFFE82EFCD7EF6A00EE47
:1040900043F010EE43F0F5EC02F000EE58F011EEB4
:1040A000E2F041500401185DEAEC02F0EF6A41527F
:1040B0000001D8A45FEF20F000EE58F0EE6A00EEA9
:1040C00058F010EE58F0F5EC02F001EE31F010EE81
:1040D00058F0400EE75204E0E6CFEEFFE82EFAD7A4
:1040E000EF6AD8960101D9A5D8860001D8B68AEF23
:1040F00020F00D0EF76E9C0EF66ED7EC01F0040E5C
:10410000016E4150CCEC00F00D0EDFEC01F00A0E18
:10411000DFEC01F0D8960101D9A5D8860001D8B608
:10412000A5EF20F00D0EF76EAA0EF66ED7EC01F09B
:1041300000EE43F0EE5003E0DFEC01F0FBD70D0E94
:10414000DFEC01F00A0EDFEC01F0D8960101D9A5F1
:10415000D8860001D8B6C0EF20F00D0EF76EB80E6D
:10416000F66ED7EC01F000EE58F0EE5003E0DFEC15
:1041700001F0FBD70D0EDFEC01F00A0EDFEC01F0D1
:104180000D0EF76EC60EF66E00EE43F001EC03F076
:10419000D8A4CFEF20F0C6EC39F04AEF26F00D0E90
:1041A000F76ECE0EF66E00EE43F001EC03F0D8A4ED
:1041B000DEEF20F052EC41F04AEF26F00D0EF76EE4
:1041C000D80EF66E00EE43F001EC03F0D8A4EDEF4C
:1041D00020F078EC41F04AEF26F00D0EF76EE20E7B
:1041E000F66E00EE43F001EC03F0D8A4FCEF20F0F3
:1041F0009EEC41F04AEF26F00D0EF76EEC0EF66ED7
:1042000000EE43F001EC03F0D8A40BEF21F0C4EC76
:1042100041F04AEF26F00D0EF76EF60EF66E00EE48
:1042200043F001EC03F0D8A41AEF21F0EAEC41F0DE
:104230004AEF26F00E0EF76E000EF66E00EE43F01B
:1042400001EC03F0D8A429EF21F010EC42F04AEF82
:1042500026F00E0EF76E0A0EF66E00EE43F001EC3D
:1042600003F0D8A438EF21F036EC42F04AEF26F004
:104270000E0EF76E140EF66E00EE43F001EC03F036
:10428000D8A447EF21F05CEC42F04AEF26F00E0E86
:10429000F76E1E0EF66E00EE43F001EC03F0D8A4AC
:1042A00056EF21F082EC42F04AEF26F00E0EF76E48
:1042B000280EF66E00EE43F001EC03F0D8A465EF93
:1042C00021F0A8EC42F04AEF26F00E0EF76E320E07
:1042D000F66E00EE43F001EC03F0D8A474EF21F089
:1042E000CEEC42F04AEF26F00E0EF76E3A0EF66E66
:1042F00000EE43F001EC03F0D8A483EF21F034EC9E
:1043000043F04AEF26F00E0EF76E420EF66E00EE08
:1043100043F001EC03F0D8A49EEF21F006011189CF
:1043200004EEA5F00E0EF76E4C0EF66ED9EC02F010
:10433000EF6A0001E4EC1DF04AEF26F00E0EF76E76
:10434000620EF66E00EE43F001EC03F0D8A4B9EF74
:1043500021F00601119904EEA5F00E0EF76E6C0E19
:10436000F66ED9EC02F0EF6A0001E4EC1DF04AEFC2
:1043700026F00E0EF76E820EF66E00EE43F001ECA4
:1043800003F0D8A4D4EF21F00601118B04EEA5F0C0
:104390000E0EF76E8C0EF66ED9EC02F0EF6A00018D
:1043A000E4EC1DF04AEF26F00E0EF76EA20EF66E4C
:1043B00000EE43F001EC03F0D8A4EFEF21F006018A
:1043C000119B04EEA5F00E0EF76EAE0EF66ED9EC54
:1043D00002F0EF6A0001E4EC1DF04AEF26F00E0E49
:1043E000F76EC60EF66E00EE43F001EC03F0D8A4B3
:1043F000FEEF21F09AEC43F04AEF26F00E0EF76E36
:10440000CC0EF66E00EE43F001EC03F0D8A40DEFF5
:1044100022F0CFEC43F04AEF26F00E0EF76ED20EEC
:10442000F66E00EE43F001EC03F0D8A41CEF22F08E
:1044300004EC44F04AEF26F00E0EF76ED80EF66E3E
:1044400000EE43F001EC03F0D8A42BEF22F039EC9E
:1044500044F04AEF26F00E0EF76EDE0EF66E00EE1A
:1044600043F001EC03F0D8A43AEF22F06EEC44F0F4
:104470004AEF26F00E0EF76EE40EF66E00EE43F0F5
:1044800001EC03F0D8A449EF22F0A3EC44F04AEF8A
:1044900026F00E0EF76EE80EF66E00EE43F001EC1D
:1044A00003F0D8A458EF22F0A3EC44F04AEF26F032
:1044B0000E0EF76EEC0EF66E00EE43F001EC03F01C
:1044C000D8A467EF22F0E9EC44F04AEF26F00E0E94
:1044D000F76EF00EF66E00EE43F001EC03F0D8A498
:1044E00076EF22F075EC45F04AEF26F00E0EF76EEF
:1044F000F60EF66E00EE43F001EC03F0D8A485EF63
:1045000022F00AEC2CF04AEF26F00E0EF76EFA0EAF
:10451000F66E00EE43F001EC03F0D8A494EF22F025
:1045200019EC2CF04AEF26F00E0EF76EFE0EF66E2A
:1045300000EE43F001EC03F0D8A4A3EF22F03DEC31
:104540002CF04AEF26F00F0EF76E040EF66E00EE1A
:1045500043F001EC03F0D8A4B2EF22F067EC2CF0AA
:104560004AEF26F00F0EF76E080EF66E00EE43F0DF
:1045700001EC03F0D8A4C1EF22F0DDEC39F04AEFF2
:1045800026F00F0EF76E100EF66E00EE43F001EC03
:1045900003F0D8A4D0EF22F015EC3AF04AEF26F061
:1045A0000F0EF76E180EF66E00EE43F001EC03F0FE
:1045B000D8A4DFEF22F04DEC3AF04AEF26F00F0ED0
:1045C000F76E200EF66E00EE43F001EC03F0D8A477
:1045D000EEEF22F085EC3AF04AEF26F00F0EF76E80
:1045E000280EF66E00EE43F001EC03F0D8A4FDEFC8
:1045F00022F086EC3AF04AEF26F00F0EF76E300EFE
:10460000F66E00EE43F001EC03F0D8A40CEF23F0BB
:1046100087EC3AF04AEF26F00F0EF76E380EF66E82
:1046200000EE43F001EC03F0D8A41BEF23F088EC7C
:104630003AF04AEF26F00F0EF76E400EF66E00EEDF
:1046400043F001EC03F0D8A42AEF23F047EC38F054
:104650004AEF26F00F0EF76E440EF66E00EE43F0B2
:1046600001EC03F0D8A439EF23F0F3EC38F04AEF73
:1046700026F00F0EF76E4C0EF66E00EE43F001ECD6
:1046800003F0D8A448EF23F0C2EC32F04AEF26F052
:104690000F0EF76E540EF66E00EE43F001EC03F0D1
:1046A000D8A457EF23F0FDEC32F04AEF26F00F0EBE
:1046B000F76E5C0EF66E00EE43F001EC03F0D8A44A
:1046C00066EF23F038EC33F04AEF26F00F0EF76E6A
:1046D000640EF66E00EE43F001EC03F0D8A475EF23
:1046E00023F073EC33F04AEF26F00F0EF76E6C0EEA
:1046F000F66E00EE43F001EC03F0D8A484EF23F053
:10470000AEEC33F04AEF26F00F0EF76E740EF66E35
:1047100000EE43F001EC03F0D8A493EF23F0E9ECB2
:1047200033F04AEF26F00F0EF76E7C0EF66E00EEB9
:1047300043F001EC03F0D8A4A2EF23F024EC34F012
:104740004AEF26F00F0EF76E840EF66E00EE43F081
:1047500001EC03F0D8A4B1EF23F05FEC34F04AEFA2
:1047600026F00F0EF76E8C0EF66E00EE43F001ECA5
:1047700003F0D8A4C0EF23F08DEC32F04AEF26F01E
:104780000F0EF76E940EF66E00EE43F001EC03F0A0
:10479000D8A4CFEF23F09AEC34F04AEF26F00F0EB6
:1047A000F76E9C0EF66E00EE43F001EC03F0D8A419
:1047B000DEEF23F0EFEC34F04AEF26F00F0EF76E49
:1047C000A40EF66E00EE43F001EC03F0D8A4EDEF7A
:1047D00023F044EC35F04AEF26F00F0EF76EAC0EE6
:1047E000F66E00EE43F001EC03F0D8A4FCEF23F0EA
:1047F00099EC35F04AEF26F00F0EF76EB40EF66E18
:1048000000EE43F001EC03F0D8A40BEF24F0E3EC4E
:1048100040F04AEF26F00F0EF76EBC0EF66E00EE7B
:1048200043F001EC03F0D8A41AEF24F001EC41F0BE
:104830004AEF26F00F0EF76EC60EF66E00EE43F04E
:1048400001EC03F0D8A429EF24F090EC2BF04AEF10
:1048500026F00F0EF76ECA0EF66E00EE43F001EC76
:1048600003F0D8A438EF24F088EC2BF04AEF26F0C0
:104870000F0EF76ED00EF66E00EE43F001EC03F073
:10488000D8A447EF24F0EFEC52F04AEF26F00F0ED9
:10489000F76ED60EF66E00EE43F001EC03F0D8A4EE
:1048A00056EF24F0D8EC49F04AEF26F00F0EF76EE1
:1048B000DC0EF66E00EE43F001EC03F0D8A465EFD9
:1048C00024F064EC46F04AEF26F00F0EF76EE20E8D
:1048D000F66E00EE43F001EC03F0D8A474EF24F080
:1048E00093EC4DF04AEF26F00F0EF76EEA0EF66EDF
:1048F00000EE43F001EC03F0D8A483EF24F009ECC0
:1049000027F04AEF26F00F0EF76EF00EF66E00EE6F
:1049100043F001EC03F0D8A492EF24F027EC2AF046
:104920004AEF26F00F0EF76EF80EF66E00EE43F02B
:1049300001EC03F0D8A4ADEF24F00101D98104EE1D
:10494000A5F0100EF76E000EF66ED9EC02F0EF6ACD
:104950000001E4EC1DF04AEF26F0100EF76E0E0E8B
:10496000F66E00EE43F001EC03F0D8A4C8EF24F09B
:104970000101D99104EEA5F0100EF76E180EF66E37
:10498000D9EC02F0EF6A0001E4EC1DF04AEF26F0EA
:10499000100EF76E280EF66E00EE43F001EC03F0F9
:1049A000D8A4E3EF24F00101D98304EEA5F0100EA2
:1049B000F76E320EF66ED9EC02F0EF6A0001E4EC0D
:1049C0001DF04AEF26F0100EF76E500EF66E00EE58
:1049D00043F001EC03F0D8A4FEEF24F00101D993D9
:1049E00004EEA5F0100EF76E5C0EF66ED9EC02F038
:1049F000EF6A0001E4EC1DF04AEF26F0100EF76EAE
:104A00007A0EF66E00EE43F001EC03F0D8A419EF35
:104A100025F00101D98504EEA5F0100EF76E860E83
:104A2000F66ED9EC02F0EF6A0001E4EC1DF04AEFFB
:104A300026F0100EF76E9C0EF66E00EE43F001ECC1
:104A400003F0D8A434EF25F00101D99504EEA5F0C8
:104A5000100EF76EA80EF66ED9EC02F0EF6A0001A8
:104A6000E4EC1DF04AEF26F0100EF76EC00EF66E65
:104A700000EE43F001EC03F0D8A443EF25F051EC35
:104A800026F04AEF26F0100EF76EC60EF66E00EE18
:104A900043F001EC03F0D8A452EF25F084EC26F0AB
:104AA0004AEF26F0100EF76ED00EF66E00EE43F0D1
:104AB00001EC03F0D8A461EF25F00EEC2BF04AEFE7
:104AC00026F0100EF76EDA0EF66E00EE43F001ECF3
:104AD00003F0D8A470EF25F0B6EC2BF04AEF26F0E7
:104AE000100EF76EE40EF66E00EE43F001EC03F0EC
:104AF000D8A47FEF25F0B6EC2BF04AEF26F0100E8D
:104B0000F76EE80EF66E00EE43F001EC03F0D8A469
:104B10009AEF25F00401A46B04EEA5F0100EF76ED9
:104B2000F20EF66ED9EC02F0EF6A0001E4EC1DF033
:104B30004AEF26F0110EF76E0E0EF66E00EE43F001
:104B400001EC03F0D8A4B6EF25F0010E0401A46F28
:104B500004EEA5F0110EF76E160EF66ED9EC02F00B
:104B6000EF6A0001E4EC1DF04AEF26F0110EF76E3B
:104B7000400EF66E00EE43F001EC03F0D8A4C5EF52
:104B800025F020EC1CF04AEF26F0110EF76E460ED1
:104B9000F66E00EE43F001EC03F0D8A4D4EF25F05C
:104BA00098EC2BF04AEF26F0110EF76E540EF66ECD
:104BB00000EE43F001EC03F0D8A4E3EF25F0B5ECF0
:104BC00045F04AEF26F0110EF76E5A0EF66E00EE23
:104BD00043F001EC03F0D8A4F2EF25F01DEF15F03F
:104BE0004AEF26F0110EF76E620EF66E00EE43F0FD
:104BF00001EC03F0D8A401EF26F01FEC41F04AEFDE
:104C000026F0110EF76E6A0EF66E00EE43F001EC20
:104C100003F0D8A410EF26F034EC41F04AEF26F070
:104C2000110EF76E720EF66E00EE43F001EC03F01B
:104C3000D8A41FEF26F0CBEC31F04AEF26F0110E8E
:104C4000F76E760EF66E00EE43F001EC03F0D8A49A
:104C50002EEF26F06CEC40F04AEF26F0110EF76EC6
:104C60007E0EF66E00EE43F001EC03F0D8A43DEFAB
:104C700026F090EC40F04AEF26F0110EF76E840E0D
:104C8000F66E00EE43F001EC03F0D8A44AEF26F0F4
:104C900029EC40F00401A36BA26B0001E9EC17F0D2
:104CA000120002EECBF0110EF76E8A0EF66ED9EC02
:104CB00002F011EEDCF0040EE75204E0E6CFEEFF66
:104CC000E82EFAD7110EF76E920EF66ED9EC02F0BE
:104CD00015EEE4F0060EE75204E0E6CFEEFFE82E14
:104CE000FAD7110EF76E9C0EF66ED9EC02F0020E9A
:104CF000016E0501ED51CCEC00F0EF6A000131ECE2
:104D00001CF0D9EC1EF012000501ED510A0DF3CF95
:104D10001CF0F4CF1DF026EC02F00001C2DF1200FF
:104D20000401A4530001D8A4CAEF26F002EECBF090
:104D3000110EF76EA80EF66ED9EC02F0020E016E9F
:104D4000E86A82B8010ECCEC00F0020E016EE86A4F
:104D500082BA010ECCEC00F0020E016EE86A81B05E
:104D6000010ECCEC00F0020E016EE86A81B2010E79
:104D7000CCEC00F0020E016EE86A81B4010ECCECBE
:104D800000F0300EEE6EEE6EEE6EEF6A31EC1CF05F
:104D9000D9EC1EF0010E0401A45D0001D8A405EFBA
:104DA00027F002EECBF0110EF76EB00EF66ED9ECD6
:104DB00002F0020E016EE86A82B8010ECCEC00F03F
:104DC000020E016EE86A82BA010ECCEC00F0020E0F
:104DD000016EE86A81B0010ECCEC00F0020E016EAB
:104DE000E86A81B2010ECCEC00F0020E016EE86AB6
:104DF00081B4010ECCEC00F0300EEE6EEE6EEE6E75
:104E0000EF6A31EC1CF0D9EC1EF0140E24EC02F029
:104E100012000401A4530001D8A497EF28F002EE79
:104E2000CBF0110EF76EB80EF66ED9EC02F0020E52
:104E3000016EE86A82B8010ECCEC00F0020E016E41
:104E4000E86A82BA010ECCEC00F0020E016EE86A4C
:104E500081B0010ECCEC00F0020E016EE86A81B266
:104E6000010ECCEC00F0020E016EE86A81B4010E76
:104E7000CCEC00F0300EEE6EEE6EEE6EEF6A31ECC2
:104E80001CF0D9EC1EF0140E24EC02F002EECBF074
:104E9000110EF76EC00EF66ED9EC02F0020E016E26
:104EA0003BC52FF03AC52EF039C52DF038C52CF092
:104EB000030EFEEC00F02C0EEE6E020E016E3FC5EE
:104EC0002FF03EC52EF03DC52DF03CC52CF0030E55
:104ED000FEEC00F02C0EEE6E020E016E43C52FF0BC
:104EE00042C52EF041C52DF040C52CF0030EFEEC5E
:104EF00000F02C0EEE6E020E016E47C52FF046C577
:104F00002EF045C52DF044C52CF0030EFEEC00F04C
:104F1000EF6A31EC1CF0D9EC1EF0140E24EC02F018
:104F200002EECBF0110EF76EC80EF66ED9EC02F061
:104F3000020E016E086AF6C521F0F5C520F0CFEC2F
:104F400000F02C0EEE6E020E016E086AF8C521F01C
:104F5000F7C520F0CFEC00F02C0EEE6E020E016EC5
:104F6000086AFAC521F0F9C520F0CFEC00F02C0E4C
:104F7000EE6E020E016E086AFCC521F0FBC520F042
:104F8000CFEC00F02C0EEE6E020E016E086AFEC52C
:104F900021F0FDC520F0CFEC00F02C0EEE6E020EDD
:104FA000016E086A00C621F0FFC520F0CFEC00F0CA
:104FB0002C0EEE6E020E016E086A02C621F001C6CA
:104FC00020F0CFEC00F02C0EEE6E020E016E000E03
:104FD000CCEC00F02C0EEE6E020E016EE86A0601BB
:104FE00011B9010ECCEC00F0EF6A000131EC1CF0BD
:104FF000D9EC1EF0140E24EC02F002EECBF0110EF0
:10500000F76ED00EF66ED9EC02F0020E016E086A51
:1050100004C621F003C620F0CFEC00F02C0EEE6E9B
:10502000020E016E086A06C621F005C620F0CFEC1C
:1050300000F02C0EEE6E020E016E086A08C621F01A
:1050400007C620F0CFEC00F02C0EEE6E020E016EC3
:10505000086A0AC621F009C620F0CFEC00F02C0E39
:10506000EE6E020E016E086A0CC621F00BC620F02F
:10507000CFEC00F02C0EEE6E020E016E086A0EC62A
:1050800021F00DC620F0CFEC00F02C0EEE6E020EDB
:10509000016E086A10C621F00FC620F0CFEC00F0B8
:1050A0002C0EEE6E020E016E000ECCEC00F02C0EFB
:1050B000EE6E020E016EE86A060111BB010ECCEC29
:1050C00000F0EF6A000131EC1CF0D9EC1EF0140E78
:1050D00024EC02F002EECBF0110EF76ED80EF66E55
:1050E000D9EC02F0020E016E0501ED51CCEC00F09E
:1050F0002C0EEE6E020E016E086AE1C521F0E0C5CD
:1051000020F0CFEC00F02C0EEE6E020E016E086A5D
:10511000E3C521F0E2C520F0CFEC00F0EF6A00011A
:1051200031EC1CF0D9EC1EF0140E24EC02F0010E50
:105130000401A45D0001D8A426EF2AF002EECBF012
:10514000110EF76EE00EF66ED9EC02F0020E016E53
:10515000E86A82B8010ECCEC00F0020E016EE86A3B
:1051600082BA010ECCEC00F0020E016EE86A81B04A
:10517000010ECCEC00F0020E016EE86A81B2010E65
:10518000CCEC00F0020E016EE86A81B4010ECCECAA
:1051900000F0300EEE6EEE6EEE6EEF6A31EC1CF04B
:1051A000D9EC1EF0140E24EC02F002EECBF0110E3E
:1051B000F76EE80EF66ED9EC02F0020E016E3BC5FA
:1051C0002FF03AC52EF039C52DF038C52CF0030E5E
:1051D000FEEC00F02C0EEE6E020E016E3FC52FF0BD
:1051E0003EC52EF03DC52DF03CC52CF0030EFEEC67
:1051F00000F02C0EEE6E020E016E43C52FF042C57C
:105200002EF041C52DF040C52CF0030EFEEC00F051
:105210002C0EEE6E020E016E47C52FF046C52EF025
:1052200045C52DF044C52CF0030EFEEC00F0EF6AEE
:1052300031EC1CF0D9EC1EF0140E24EC02F002EE5E
:10524000CBF0110EF76EF00EF66ED9EC02F0020EF6
:10525000016E086AF6C521F0F5C520F0CFEC00F02C
:105260002C0EEE6E020E016E086AF8C521F0F7C52D
:1052700020F0CFEC00F02C0EEE6E020E016E086AEC
:10528000FAC521F0F9C520F0CFEC00F02C0EEE6E3F
:10529000020E016E086AFCC521F0FBC520F0CFECC0
:1052A00000F02C0EEE6E020E016E086AFEC521F0B3
:1052B000FDC520F0CFEC00F02C0EEE6E020E016E5C
:1052C000086A00C621F0FFC520F0CFEC00F02C0EDC
:1052D000EE6E020E016E086A02C621F001C620F0D1
:1052E000CFEC00F02C0EEE6E020E016E000ECCEC38
:1052F00000F02C0EEE6E020E016EE86A060111B986
:10530000010ECCEC00F0EF6A000131EC1CF0D9EC9E
:105310001EF0140E24EC02F002EECBF0110EF76E2C
:10532000F80EF66ED9EC02F0020E016E086A04C6A1
:1053300021F003C620F0CFEC00F02C0EEE6E020E32
:10534000016E086A06C621F005C620F0CFEC00F019
:105350002C0EEE6E020E016E086A08C621F007C61A
:1053600020F0CFEC00F02C0EEE6E020E016E086AFB
:105370000AC621F009C620F0CFEC00F02C0EEE6E2C
:10538000020E016E086A0CC621F00BC620F0CFECAD
:1053900000F02C0EEE6E020E016E086A0EC621F0B1
:1053A0000DC620F0CFEC00F02C0EEE6E020E016E5A
:1053B000086A10C621F00FC620F0CFEC00F02C0ECA
:1053C000EE6E020E016E000ECCEC00F02C0EEE6EB6
:1053D000020E016EE86A060111BB010ECCEC00F072
:1053E000EF6A000131EC1CF0D9EC1EF0140E24EC35
:1053F00002F002EECBF0120EF76E000EF66ED9EC54
:1054000002F0020E016E0501ED51CCEC00F02C0E05
:10541000EE6E020E016E086AE1C521F0E0C520F0D3
:10542000CFEC00F02C0EEE6E020E016E086AE3C5A2
:1054300021F0E2C520F0CFEC00F0EF6A000131EC82
:105440001CF0D9EC1EF0140E24EC02F0120002EE57
:10545000CBF0120EF76E080EF66ED9EC02F0020ECB
:10546000016EE86A82B8010ECCEC00F0020E016E0B
:10547000E86A82BA010ECCEC00F0020E016EE86A16
:1054800081B0010ECCEC00F0020E016EE86A81B230
:10549000010ECCEC00F0020E016EE86A81B4010E40
:1054A000CCEC00F0300EEE6EEE6EEE6E2C0EEE6E6C
:1054B000020E016E3BC52FF03AC52EF039C52DF016
:1054C00038C52CF0030EFEEC00F02C0EEE6E020E32
:1054D000016E3FC52FF03EC52EF03DC52DF03CC5F9
:1054E0002CF0030EFEEC00F02C0EEE6E020E016EA0
:1054F00043C52FF042C52EF041C52DF040C52CF01C
:10550000030EFEEC00F02C0EEE6E020E016E47C58F
:105510002FF046C52EF045C52DF044C52CF0030EE6
:10552000FEEC00F02C0EEE6E020E016EE86A80BA00
:10553000010ECCEC00F0020E016EE86A81B6010E9D
:10554000CCEC00F0020E016EE86A81B8010ECCECE2
:1055500000F0020E016EE86A82B6010ECCEC00F09B
:10556000EF6A31EC1CF0D9EC1EF0140E24EC02F0C2
:105570001200120EF76E100EF66E01EEDCF001EC6A
:1055800003F0D8A4E0EF2AF0010E0101CC6F000176
:10559000040E0101CC5D0001D8B0DEEF2AF0949238
:1055A0008292FA0E24EC02F094928282FA0E24EC9B
:1055B00002F00101CC2B0001D8A4E9D70DEF2BF0AC
:1055C000010E0101CC6F0001030E0101CC5D000151
:1055D000D8B00DEF2BF094928292010E1D6EF40E56
:1055E00025EC02F094928282C80E24EC02F0949290
:1055F0008292010E1D6EF40E25EC02F094928282CE
:10560000C80E24EC02F0010E1D6E900E25EC02F087
:105610000101CC2B0001D8A4D6D7120001EEDCF09A
:10562000460EEE6E410EEE6E490EEE6E4C0EEE6EB6
:10563000EF6A120081EC2BF001EE31F0120EF76EE2
:10564000140EF66ED9EC02F0020E016E0501ED515A
:10565000CCEC00F0120EF76E280EF66ED9EC02F0CC
:10566000EF6A000120EC1CF0010E0101CC6F00017B
:10567000040E0101CC5D0001D8B064EF2BF09492D0
:105680008292820E026E040E096E010E046EF40EFA
:10569000036E030E216EE80E206E33EC00F0949240
:1056A0008282820E026E040E096E010E046EF40EEA
:1056B000036E010E216E900E206E33EC00F001019E
:1056C000CC2B0001D8A4D3D705EE93F0460EEE6E96
:1056D000410EEE6E490EEE6E4C0EEE6EEF6A89ECE8
:1056E0002CF094928292010E1D6EF40E25EC02F0C5
:1056F00094928282010E1D6EF40E25EC02F0F1D719
:1057000012008298829A81908192819412001200F4
:105710000501266B01016B6B060111970001120058
:10572000010E0501266F010E01016B6F00011200D1
:1057300001EE31F084EC00F00501F36F21C0F4F5C7
:1057400004EEA5F0120EF76E3A0EF66ED9EC02F0EA
:10575000020E016E086AF4C521F0F3C520F0CFEC0B
:1057600000F0EF6A0001E4EC1DF01200CADF2D0E1C
:105770000101CC6F010ED46F0001090E0101D45D4F
:105780000001D8B008EF2CF0949882880101CC5128
:1057900024EC02F094988298949A828ACC5124EC5A
:1057A00002F0949A829A93908180CC5124EC02F07A
:1057B0009390819093928182CC5124EC02F0939249
:1057C000819293948184CC5124EC02F0939481943F
:1057D00093928182CC5124EC02F093928192939027
:1057E0008180CC5124EC02F093908190949A828A2B
:1057F000CC5124EC02F0949A829A94988288CC51ED
:1058000024EC02F094988298D42B0001D8A4B4D749
:1058100078DF120005EE93F011EE31F0360EE7520C
:1058200004E0E6CFEEFFE82EFAD7EF6A89EC2CF021
:10583000120093928182C80E24EC02F005EE93F0E0
:1058400011EE31F0360EE75204E0E6CFEEFFE82E1F
:10585000FAD7EF6A89EC2CF0640E24EC02F09392F4
:10586000819204EEA5F0120EF76E540EF66ED9EC8E
:1058700002F0EF6AE4EC1DF01200120EF76E5C0EFF
:10588000F66E01EE31F001EC03F0D8A458EF2CF0E5
:1058900005012B8504EEA5F0120EF76E600EF66E74
:1058A000D9EC02F0EF6A0001E4EC1DF066EF2CF099
:1058B00005012B9504EEA5F0120EF76E6E0EF66E36
:1058C000D9EC02F0EF6A0001E4EC1DF0120001EEE9
:1058D00031F084EC00F00501916F040E196EB00EEA
:1058E000186E1D6A91C51CF09CEC02F08F6F19C0F8
:1058F00090F504EEA5F0120EF76E7E0EF66ED9EC62
:1059000002F0020E016E9151CCEC00F0EF6A000142
:10591000120004EEA5F0120EF76E900EF66ED9ECA2
:1059200002F015EE93F0320EE75204E0E6CFEEFF00
:10593000E82EFAD7EF6AE4EC1DF0040E196EB00EF3
:10594000186E1D6A91C51CF09CEC02F005018F6F6A
:1059500019C090F59492828205EE93F0E86AEE52B7
:1059600002E0E83EFCD7926F010E0101CC6F00010E
:105970000101CC510501925D0001D8A083EF2FF009
:1059800005EEC6F015EE93F0CCC1F3FF010EE1EC8D
:1059900002F0EF6A410E0501C65D0001D8A4DAEFFE
:1059A0002CF005EECBF02E0EEE6E2D0EEE6EEF6AA5
:1059B0007BEF2FF0420E0501C65D0001D8A4ECEF8D
:1059C0002CF005EECBF02D0EEE6E2E0EEE6EEE6E82
:1059D000EE6EEF6A7BEF2FF0430E0501C65D00010E
:1059E000D8A400EF2DF005EECBF02D0EEE6E2E0EAE
:1059F000EE6E2D0EEE6E2E0EEE6EEF6A7BEF2FF03A
:105A0000440E0501C65D0001D8A411EF2DF005EE8E
:105A1000CBF02D0EEE6E2E0EEE6EEE6EEF6A7BEF7D
:105A20002FF0450E0501C65D0001D8A41FEF2DF033
:105A300005EECBF02E0EEE6EEF6A7BEF2FF0460EEA
:105A40000501C65D0001D8A432EF2DF005EECBF0C4
:105A50002E0EEE6EEE6E2D0EEE6E2E0EEE6EEF6ACA
:105A60007BEF2FF0470E0501C65D0001D8A443EF80
:105A70002DF005EECBF02D0EEE6EEE6E2E0EEE6ED0
:105A8000EF6A7BEF2FF0480E0501C65D0001D8A438
:105A900054EF2DF005EECBF02E0EEE6EEE6EEE6EA8
:105AA000EE6EEF6A7BEF2FF0490E0501C65D000137
:105AB000D8A463EF2DF005EECBF02E0EEE6EEE6E59
:105AC000EF6A7BEF2FF04A0E0501C65D0001D8A4F6
:105AD00075EF2DF005EECBF02E0EEE6E2D0EEE6E68
:105AE000EE6EEE6EEF6A7BEF2FF04B0E0501C65D9A
:105AF0000001D8A487EF2DF005EECBF02D0EEE6E51
:105B00002E0EEE6E2D0EEE6EEF6A7BEF2FF04C0E2A
:105B10000501C65D0001D8A49AEF2DF005EECBF08B
:105B20002E0EEE6E2D0EEE6E2E0EEE6EEE6EEF6AF9
:105B30007BEF2FF04D0E0501C65D0001D8A4A9EF43
:105B40002DF005EECBF02D0EEE6EEE6EEF6A7BEFD4
:105B50002FF04E0E0501C65D0001D8A4B9EF2DF05F
:105B600005EECBF02D0EEE6E2E0EEE6EEF6A7BEF95
:105B70002FF04F0E0501C65D0001D8A4C9EF2DF02E
:105B800005EECBF02D0EEE6EEE6EEE6EEF6A7BEF55
:105B90002FF0500E0501C65D0001D8A4DCEF2DF0FA
:105BA00005EECBF02E0EEE6E2D0EEE6EEE6E2E0E80
:105BB000EE6EEF6A7BEF2FF0510E0501C65D00011E
:105BC000D8A4EFEF2DF005EECBF02D0EEE6EEE6EBD
:105BD0002E0EEE6E2D0EEE6EEF6A7BEF2FF0520E54
:105BE0000501C65D0001D8A401EF2EF005EECBF053
:105BF0002E0EEE6E2D0EEE6E2E0EEE6EEF6A7BEF1B
:105C00002FF0530E0501C65D0001D8A411EF2EF050
:105C100005EECBF02E0EEE6EEE6EEE6EEF6A7BEFC3
:105C20002FF0540E0501C65D0001D8A41FEF2EF021
:105C300005EECBF02D0EEE6EEF6A7BEF2FF0550EDA
:105C40000501C65D0001D8A430EF2EF005EECBF0C3
:105C50002E0EEE6EEE6E2D0EEE6EEF6A7BEF2FF0D7
:105C6000560E0501C65D0001D8A442EF2EF005EEE8
:105C7000CBF02E0EEE6EEE6EEE6E2D0EEE6EEF6A29
:105C80007BEF2FF0570E0501C65D0001D8A453EF3E
:105C90002EF005EECBF02E0EEE6E2D0EEE6EEE6EAD
:105CA000EF6A7BEF2FF0580E0501C65D0001D8A406
:105CB00066EF2EF005EECBF02D0EEE6E2E0EEE6E94
:105CC000EE6E2D0EEE6EEF6A7BEF2FF0590E050192
:105CD000C65D0001D8A479EF2EF005EECBF02D0EB5
:105CE000EE6E2E0EEE6E2D0EEE6EEE6EEF6A7BEF0A
:105CF0002FF05A0E0501C65D0001D8A48BEF2EF0DF
:105D000005EECBF02D0EEE6EEE6E2E0EEE6EEE6EFE
:105D1000EF6A7BEF2FF0300E0501C65D0001D8A4BD
:105D20009DEF2EF005EECBF02D0EEE6EEE6EEE6ECC
:105D3000EE6EEE6EEF6A7BEF2FF0310E0501C65D61
:105D40000001D8A4B0EF2EF005EECBF02E0EEE6ED3
:105D50002D0EEE6EEE6EEE6EEE6EEF6A7BEF2FF0B6
:105D6000320E0501C65D0001D8A4C3EF2EF005EE8A
:105D7000CBF02E0EEE6EEE6E2D0EEE6EEE6EEE6E25
:105D8000EF6A7BEF2FF0330E0501C65D0001D8A44A
:105D9000D6EF2EF005EECBF02E0EEE6EEE6EEE6E22
:105DA0002D0EEE6EEE6EEF6A7BEF2FF0340E0501D6
:105DB000C65D0001D8A4E8EF2EF005EECBF02E0E64
:105DC000EE6EEE6EEE6E2D0EEE6EEF6A7BEF2FF046
:105DD000350E0501C65D0001D8A4FAEF2EF005EEE0
:105DE000CBF02E0EEE6EEE6EEE6EEE6EEE6EEF6A97
:105DF0007BEF2FF0360E0501C65D0001D8A40DEF34
:105E00002FF005EECBF02D0EEE6E2E0EEE6EEE6E3A
:105E1000EE6EEE6EEF6A7BEF2FF0370E0501C65D7A
:105E20000001D8A420EF2FF005EECBF02D0EEE6E82
:105E3000EE6E2E0EEE6EEE6EEE6EEF6A7BEF2FF0D4
:105E4000380E0501C65D0001D8A433EF2FF005EE32
:105E5000CBF02D0EEE6EEE6EEE6E2E0EEE6EEE6E44
:105E6000EF6A7BEF2FF0390E0501C65D0001D8A463
:105E700046EF2FF005EECBF02D0EEE6EEE6EEE6ED1
:105E8000EE6E2E0EEE6EEF6A7BEF2FF02F0E0501F9
:105E9000C65D0001D8A45BEF2FF005EECBF02D0E10
:105EA000EE6E2E0EEE6EEE6E2D0EEE6E2E0EEE6E73
:105EB000EF6A7BEF2FF03D0E0501C65D0001D8A40F
:105EC0006FEF2FF005EECBF02D0EEE6E2E0EEE6E78
:105ED000EE6EEE6E2D0EEE6EEF6A7BEF2FF0200E63
:105EE0000501C65D0001D8A47BEF2FF005EECBF0D5
:105EF000200EEE6EEF6A84EC2FF00101CC2B000136
:105F0000D8A4B7EF2CF0120005EECBF0E86AEE5201
:105F100002E0E83EFCD70101D46F010ED76F00010B
:105F20000101D751D45D0001D8A01DEF30F005EE7E
:105F3000C8F015EECBF0D7C1F3FF010EE1EC02F093
:105F4000EF6A2E0E0501C85D0001D8A4CCEF2FF03A
:105F5000D89605012BA5D8860001D8B6B2EF2FF050
:105F600093948184820E026E040E096E90C504F033
:105F70008FC503F08EC521F08DC520F033EC00F005
:105F8000D89605012BA5D8860001D8B6CAEF2FF008
:105F90009394819412EF30F02D0E0501C85D00013D
:105FA000D8A4FDEF2FF0D89605012BA5D8860001C7
:105FB000D8B6DDEF2FF093948184820E026E040E2A
:105FC000096E05019051030DF3CF04F08F51030DBD
:105FD000F3CF03F0F45004268EC521F08DC520F0D8
:105FE00033EC00F0D8962BA5D8860001D8B6FBEF8D
:105FF0002FF09394819412EF30F0200E0501C85DCC
:106000000001D8A411EF30F005019051030DF3CF3A
:106010001DF08F51030DF3CF1CF0F4501D2626EC1C
:1060200002F0000190C51DF005018F5125EC02F032
:106030000101D72B0001D8A472D705019051030D9F
:10604000F3CF1DF08F51030DF3CF1CF0F4501D263C
:1060500026EC02F000011200000E0DEC02F005012A
:10606000306F2DC031F5176A166A156A8F0E146EDF
:1060700031C511F030C510F0D0EC04F018EC04F08C
:1060800013C0D2F112C0D1F111C0D0F110C0CFF1C4
:10609000136A126A200E116E810E106ED2C117F0B3
:1060A000D1C116F0D0C115F0CFC114F080EC04F0CE
:1060B00013C02FF012C02EF011C02DF010C02CF024
:1060C0002FC013F02EC012F02DC011F02CC010F014
:1060D0002FC517F02EC516F02DC515F02CC514F0E0
:1060E00080EC04F013C03BF512C03AF511C039F54D
:1060F00010C038F53BC513F03AC512F039C511F0A0
:1061000038C510F04BC517F04AC516F049C515F053
:1061100048C514F07EEC03F013C03BF512C03AF50D
:1061200011C039F510C038F5010E0DEC02F0326FD8
:106130002DC033F5176A166A156A8F0E146E33C5B3
:1061400011F032C510F0D0EC04F018EC04F013C0DC
:10615000D2F112C0D1F111C0D0F110C0CFF1136A49
:10616000126A200E116E810E106ED2C117F0D1C1CD
:1061700016F0D0C115F0CFC114F080EC04F013C0BC
:106180002FF012C02EF011C02DF010C02CF02FC037
:1061900013F02EC012F02DC011F02CC010F02FC53E
:1061A00017F02EC516F02DC515F02CC514F080EC97
:1061B00004F013C03FF512C03EF511C03DF510C00C
:1061C0003CF53FC513F03EC512F03DC511F03CC58E
:1061D00010F04FC517F04EC516F04DC515F04CC563
:1061E00014F07EEC03F013C03FF512C03EF511C071
:1061F0003DF510C03CF5020E0DEC02F0346F2DC0E1
:1062000035F5176A166A156A8F0E146E35C511F0CA
:1062100034C510F0D0EC04F018EC04F013C0D2F147
:1062200012C0D1F111C0D0F110C0CFF1136A126ABF
:10623000200E116E810E106ED2C117F0D1C116F072
:10624000D0C115F0CFC114F080EC04F013C02FF0D2
:1062500012C02EF011C02DF010C02CF02FC013F082
:106260002EC012F02DC011F02CC010F02FC517F069
:106270002EC516F02DC515F02CC514F080EC04F0D9
:1062800013C043F512C042F511C041F510C040F5EE
:1062900043C513F042C512F041C511F040C510F0DE
:1062A00053C517F052C516F051C515F050C514F07E
:1062B0007EEC03F013C043F512C042F511C041F566
:1062C00010C040F5030E0DEC02F0366F2DC037F50F
:1062D000176A166A156A8F0E146E37C511F036C527
:1062E00010F0D0EC04F018EC04F013C0D2F112C09E
:1062F000D1F111C0D0F110C0CFF1136A126A200E93
:10630000116E810E106ED2C117F0D1C116F0D0C13E
:1063100015F0CFC114F080EC04F013C02FF012C0C0
:106320002EF011C02DF010C02CF02FC013F02EC095
:1063300012F02DC011F02CC010F02FC517F02EC593
:1063400016F02DC515F02CC514F080EC04F013C028
:1063500047F512C046F511C045F510C044F547C5D4
:1063600013F046C512F045C511F044C510F057C5ED
:1063700017F056C516F055C515F054C514F07EEC4F
:1063800003F013C047F512C046F511C045F510C023
:1063900044F50001120004EEA5F0120EF76E9A0EFD
:1063A000F66ED9EC02F0EF6AE4EC1DF00A0E24EC74
:1063B00002F052DE04EEA5F0120EF76EC00EF66E7D
:1063C000D9EC02F0020E016E3BC52FF03AC52EF05B
:1063D00039C52DF038C52CF0030EFEEC00F0120E7E
:1063E000F76ED00EF66ED9EC02F0020E016E086A5E
:1063F00031C521F030C520F0CFEC00F0290EEE6E53
:10640000EF6AE4EC1DF004EEA5F0120EF76EDA0E62
:10641000F66ED9EC02F0020E016E3FC52FF03EC5BC
:106420002EF03DC52DF03CC52CF0030EFEEC00F027
:10643000120EF76EEA0EF66ED9EC02F0020E016E45
:10644000086A33C521F032C520F0CFEC00F0290EE8
:10645000EE6EEF6AE4EC1DF004EEA5F0120EF76E9E
:10646000F40EF66ED9EC02F0020E016E43C52FF069
:1064700042C52EF041C52DF040C52CF0030EFEECB8
:1064800000F0130EF76E040EF66ED9EC02F0020E59
:10649000016E086A35C521F034C520F0CFEC00F05C
:1064A000290EEE6EEF6AE4EC1DF004EEA5F0130E7B
:1064B000F76E0E0EF66ED9EC02F0020E016E47C5B5
:1064C0002FF046C52EF045C52DF044C52CF0030E27
:1064D000FEEC00F0130EF76E1E0EF66ED9EC02F015
:1064E000020E016E086A37C521F036C520F0CFECE8
:1064F00000F0290EEE6EEF6AE4EC1DF004EEA5F05C
:10650000130EF76E280EF66ED9EC02F0EF6AE4EC8B
:106510001DF00A0E24EC02F01200130EF76E4E0E60
:10652000F66E01EE31F001EC03F0D8A4A7EF32F0E3
:10653000010E01016C6F04EEA5F0130EF76E520E02
:10654000F66ED9EC02F0EF6A0001E4EC1DF0130ED8
:10655000F76E6E0EF66E01EE31F001EC03F0D8A48A
:10656000C0EF32F001016C6B04EEA5F0130EF76E74
:10657000720EF66ED9EC02F0EF6A0001E4EC1DF049
:106580001200120001EE31F084EC00F020C010F097
:1065900021C011F022C012F023C013F0D2EC04F09D
:1065A00013C05BF512C05AF511C059F510C058F56B
:1065B00001EEA0F0020E016E5BC52FF05AC52EF061
:1065C00059C52DF058C52CF0030EFEEC00F0EF6A13
:1065D00004EEA5F0130EF76E8E0EF66ED9EC02F0F7
:1065E00011EEA0F0140EE75204E0E6CFEEFFE82E25
:1065F000FAD7EF6AE4EC1DF0120001EE31F084EC02
:1066000000F020C010F021C011F022C012F023C011
:1066100013F0D2EC04F013C05FF512C05EF511C0A8
:106620005DF510C05CF501EEA0F0020E016E5FC5D5
:106630002FF05EC52EF05DC52DF05CC52CF0030E6D
:10664000FEEC00F0EF6A04EEA5F0130EF76EA40E58
:10665000F66ED9EC02F011EEA0F0140EE75204E051
:10666000E6CFEEFFE82EFAD7EF6AE4EC1DF0120059
:1066700001EE31F084EC00F020C010F021C011F0E8
:1066800022C012F023C013F0D2EC04F013C063F563
:1066900012C062F511C061F510C060F501EEA0F006
:1066A000020E016E63C52FF062C52EF061C52DF09C
:1066B00060C52CF0030EFEEC00F0EF6A04EEA5F0CE
:1066C000130EF76EBA0EF66ED9EC02F011EEA0F0D2
:1066D000140EE75204E0E6CFEEFFE82EFAD7EF6A99
:1066E000E4EC1DF0120001EE31F084EC00F020C06B
:1066F00010F021C011F022C012F023C013F0D2EC30
:1067000004F013C067F512C066F511C065F510C03E
:1067100064F501EEA0F0020E016E67C52FF066C5AC
:106720002EF065C52DF064C52CF0030EFEEC00F0D4
:10673000EF6A04EEA5F0130EF76ED00EF66ED9ECEC
:1067400002F011EEA0F0140EE75204E0E6CFEEFFE7
:10675000E82EFAD7EF6AE4EC1DF0120001EE31F0FA
:1067600084EC00F020C010F021C011F022C012F023
:1067700023C013F0D2EC04F013C06BF512C06AF51D
:1067800011C069F510C068F501EEA0F0020E016EAF
:106790006BC52FF06AC52EF069C52DF068C52CF0C9
:1067A000030EFEEC00F0EF6A04EEA5F0130EF76E98
:1067B000E60EF66ED9EC02F011EEA0F0140EE752E0
:1067C00004E0E6CFEEFFE82EFAD7EF6AE4EC1DF026
:1067D000120001EE31F084EC00F020C010F021C076
:1067E00011F022C012F023C013F0D2EC04F013C059
:1067F0006FF512C06EF511C06DF510C06CF501EEAD
:10680000A0F0020E016E6FC52FF06EC52EF06DC5A3
:106810002DF06CC52CF0030EFEEC00F0EF6A04EED8
:10682000A5F0130EF76EFC0EF66ED9EC02F011EE29
:10683000A0F0140EE75204E0E6CFEEFFE82EFAD700
:10684000EF6AE4EC1DF0120001EE31F084EC00F090
:1068500020C010F021C011F022C012F023C013F0AC
:10686000D2EC04F013C073F512C072F511C071F5CB
:1068700010C070F501EEA0F0020E016E73C52FF08E
:1068800072C52EF071C52DF070C52CF0030EFEEC14
:1068900000F0EF6A04EEA5F0140EF76E120EF66E1D
:1068A000D9EC02F011EEA0F0140EE75204E0E6CFAE
:1068B000EEFFE82EFAD7EF6AE4EC1DF0120001EECD
:1068C00031F084EC00F020C010F021C011F022C0A3
:1068D00012F023C013F0D2EC04F013C077F512C00D
:1068E00076F511C075F510C074F501EEA0F0020E3A
:1068F000016E77C52FF076C52EF075C52DF074C5E5
:106900002CF0030EFEEC00F0EF6A04EEA5F0140E7E
:10691000F76E280EF66ED9EC02F011EEA0F0140E10
:10692000E75204E0E6CFEEFFE82EFAD7EF6AE4EC98
:106930001DF0120001EE31F084EC00F020C010F0E8
:1069400021C011F022C012F023C013F0D2EC04F0E9
:1069500013C0D2F112C0D1F111C0D0F110C0CFF1EB
:106960006F0E136E120E126E030E116E750E106EF8
:10697000D2C117F0D1C116F0D0C115F0CFC114F0BB
:1069800080EC04F013C04BF512C04AF511C049F574
:1069900010C048F501EEA0F0020E016E4BC52FF0BD
:1069A0004AC52EF049C52DF048C52CF0030EFEEC6B
:1069B00000F0EF6A04EEA5F0140EF76E3E0EF66ED0
:1069C000D9EC02F011EEA0F0140EE75204E0E6CF8D
:1069D000EEFFE82EFAD7EF6AE4EC1DF0120001EEAC
:1069E00031F084EC00F020C010F021C011F022C082
:1069F00012F023C013F0D2EC04F013C0D2F112C095
:106A0000D1F111C0D0F110C0CFF16F0E136E120E84
:106A1000126E030E116E750E106ED2C117F0D1C139
:106A200016F0D0C115F0CFC114F080EC04F013C003
:106A30004FF512C04EF511C04DF510C04CF501EEEA
:106A4000A0F0020E016E4FC52FF04EC52EF04DC5C1
:106A50002DF04CC52CF0030EFEEC00F0EF6A04EEB6
:106A6000A5F0140EF76E640EF66ED9EC02F011EE7E
:106A7000A0F0140EE75204E0E6CFEEFFE82EFAD7BE
:106A8000EF6AE4EC1DF0120001EE31F084EC00F04E
:106A900020C010F021C011F022C012F023C013F06A
:106AA000D2EC04F013C0D2F112C0D1F111C0D0F178
:106AB00010C0CFF16F0E136E120E126E030E116E18
:106AC000750E106ED2C117F0D1C116F0D0C115F0FD
:106AD000CFC114F080EC04F013C053F512C052F58E
:106AE00011C051F510C050F501EEA0F0020E016E7C
:106AF00053C52FF052C52EF051C52DF050C52CF0C6
:106B0000030EFEEC00F0EF6A04EEA5F0140EF76E33
:106B10008A0EF66ED9EC02F011EEA0F0140EE752D8
:106B200004E0E6CFEEFFE82EFAD7EF6AE4EC1DF0C2
:106B3000120001EE31F084EC00F020C010F021C012
:106B400011F022C012F023C013F0D2EC04F013C0F5
:106B5000D2F112C0D1F111C0D0F110C0CFF16F0E3F
:106B6000136E120E126E030E116E750E106ED2C1E0
:106B700017F0D1C116F0D0C115F0CFC114F080ECE0
:106B800004F013C057F512C056F511C055F510C0EA
:106B900054F501EEA0F0020E016E57C52FF056C558
:106BA0002EF055C52DF054C52CF0030EFEEC00F070
:106BB000EF6A04EEA5F0140EF76EB00EF66ED9EC87
:106BC00002F011EEA0F0140EE75204E0E6CFEEFF63
:106BD000E82EFAD7EF6AE4EC1DF012003BC513F083
:106BE0003AC512F039C511F038C510F05BC517F081
:106BF0005AC516F059C515F058C514F00AEC03F043
:106C00000108D8B41EEF36F0AFEC36F06BC513F0C8
:106C10006AC512F069C511F068C510F03BC517F0E0
:106C20003AC516F039C515F038C514F00AEC03F072
:106C30000108D8B41EEF36F07BEC37F03FC513F0F7
:106C40003EC512F03DC511F03CC510F05FC517F010
:106C50005EC516F05DC515F05CC514F00AEC03F0D6
:106C60000108D8B44EEF36F0E2EC36F06FC513F001
:106C70006EC512F06DC511F06CC510F03FC517F070
:106C80003EC516F03DC515F03CC514F00AEC03F006
:106C90000108D8B44EEF36F0AEEC37F043C513F030
:106CA00042C512F041C511F040C510F063C517F0A0
:106CB00062C516F061C515F060C514F00AEC03F06A
:106CC0000108D8B47EEF36F015EC37F073C513F039
:106CD00072C512F071C511F070C510F043C517F000
:106CE00042C516F041C515F040C514F00AEC03F09A
:106CF0000108D8B47EEF36F0E1EC37F047C513F069
:106D000046C512F045C511F044C510F067C517F02F
:106D100066C516F065C515F064C514F00AEC03F0FD
:106D20000108D8B4AEEF36F048EC37F077C513F071
:106D300076C512F075C511F074C510F047C517F08F
:106D400046C516F045C515F044C514F00AEC03F02D
:106D50000108D8B4AEEF36F014EC38F0120004EEAF
:106D6000A5F0140EF76ED60EF66ED9EC02F0020EF8
:106D7000016E5BC52FF05AC52EF059C52DF058C5D0
:106D80002CF0030EFEEC00F0150EF76E020EF66E00
:106D9000D9EC02F0020E016E3BC52FF03AC52EF081
:106DA00039C52DF038C52CF0030EFEEC00F0760E40
:106DB000EE6E2E0EEE6EEF6AE4EC1DF0640E24EC27
:106DC00002F0120004EEA5F0150EF76E100EF66E2E
:106DD000D9EC02F0020E016E5FC52FF05EC52EF0F9
:106DE0005DC52DF05CC52CF0030EFEEC00F0150E19
:106DF000F76E3C0EF66ED9EC02F0020E016E3FC546
:106E00002FF03EC52EF03DC52DF03CC52CF0030EF5
:106E1000FEEC00F0760EEE6E2E0EEE6EEF6AE4ECF7
:106E20001DF0640E24EC02F0120004EEA5F0150E25
:106E3000F76E4A0EF66ED9EC02F0020E016E63C5D3
:106E40002FF062C52EF061C52DF060C52CF0030E49
:106E5000FEEC00F0150EF76E760EF66ED9EC02F031
:106E6000020E016E43C52FF042C52EF041C52DF034
:106E700040C52CF0030EFEEC00F0760EEE6E2E0EEA
:106E8000EE6EEF6AE4EC1DF0640E24EC02F01200EA
:106E900004EEA5F0150EF76E840EF66ED9EC02F036
:106EA000020E016E67C52FF066C52EF065C52DF088
:106EB00064C52CF0030EFEEC00F0150EF76EB00E5C
:106EC000F66ED9EC02F0020E016E47C52FF046C5F2
:106ED0002EF045C52DF044C52CF0030EFEEC00F05D
:106EE000760EEE6E2E0EEE6EEF6AE4EC1DF0640E82
:106EF00024EC02F0120004EEA5F0150EF76EBE0EA3
:106F0000F66ED9EC02F0020E016E6BC52FF06AC569
:106F10002EF069C52DF068C52CF0030EFEEC00F0D4
:106F2000150EF76EEA0EF66ED9EC02F0020E016E47
:106F30003BC52FF03AC52EF039C52DF038C52CF0E1
:106F4000030EFEEC00F0760EEE6E2E0EEE6EEF6A85
:106F5000E4EC1DF0640E24EC02F0120004EEA5F047
:106F6000150EF76EF80EF66ED9EC02F0020E016EF9
:106F70006FC52FF06EC52EF06DC52DF06CC52CF0D1
:106F8000030EFEEC00F0160EF76E240EF66ED9EC32
:106F900002F0020E016E3FC52FF03EC52EF03DC53A
:106FA0002DF03CC52CF0030EFEEC00F0760EEE6EDC
:106FB0002E0EEE6EEF6AE4EC1DF0640E24EC02F08F
:106FC000120004EEA5F0160EF76E320EF66ED9EC36
:106FD00002F0020E016E73C52FF072C52EF071C55E
:106FE0002DF070C52CF0030EFEEC00F0160EF76EBF
:106FF0005E0EF66ED9EC02F0020E016E43C52FF064
:1070000042C52EF041C52DF040C52CF0030EFEEC1C
:1070100000F0760EEE6E2E0EEE6EEF6AE4EC1DF0D2
:10702000640E24EC02F0120004EEA5F0160EF76ECA
:107030006C0EF66ED9EC02F0020E016E77C52FF0E1
:1070400076C52EF075C52DF074C52CF0030EFEEC40
:1070500000F0160EF76E980EF66ED9EC02F0020EE6
:10706000016E47C52FF046C52EF045C52DF044C52D
:107070002CF0030EFEEC00F0760EEE6E2E0EEE6E91
:10708000EF6AE4EC1DF0640E24EC02F01200160E20
:10709000F76EA60EF66E01EE31F001EC03F0D8A407
:1070A00060EF38F00501786B04EEA5F0160EF76E70
:1070B000AA0EF66ED9EC02F0EF6A0001E4EC1DF0C6
:1070C000160EF76ECA0EF66E01EE31F001EC03F00B
:1070D000D8A47AEF38F0010E0501786F04EEA5F020
:1070E000160EF76ECE0EF66ED9EC02F0EF6A0001C6
:1070F000E4EC1DF0160EF76EF20EF66E01EE31F0B6
:1071000001EC03F0D8A494EF38F0020E0501786F7B
:1071100004EEA5F0160EF76EFA0EF66ED9EC02F03C
:10712000EF6A0001E4EC1DF01200010E0501785D2C
:107130000001D8A4BAEF38F03BC513F03AC512F0FD
:1071400039C511F038C510F03FC517F03EC516F02F
:107150003DC515F03CC514F042EC03F00108D8B46D
:10716000B7EF38F0060111830001B9EF38F00601DE
:1071700011930001020E0501785D0001D8A4F2EF21
:1071800038F03FC513F03EC512F03DC511F03CC5C7
:1071900010F07CC517F07BC516F07AC515F079C5DF
:1071A00014F00AEC03F0356E3FC513F03EC512F043
:1071B0003DC511F03CC510F03BC517F03AC516F0BF
:1071C00039C515F038C514F00AEC03F03510D8B401
:1071D000EFEF38F0060111830001F1EF38F00601FE
:1071E00011930001120001EE31F084EC00F020C098
:1071F00010F021C011F022C012F023C013F0D2EC25
:1072000004F013C07CF512C07BF511C07AF510C0F4
:1072100079F51200120001011B6B00019EAA13EF09
:1072200039F0AECF1BF112009EB818EF39F0FCD741
:107230001BC1ADFF1200010E0501D85D0001D8A4ED
:107240002CEF39F08288FA0E24EC02F08298010EBD
:107250001D6E2C0E25EC02F0020E0501D85D00011A
:10726000D8A434EF39F08288030E0501D85D0001FF
:10727000D8A43CEF39F08298040E0501D85D0001D6
:10728000D8A445EF39F027EC2AF0050E0501D85DAA
:107290000001D8A453EF39F08278949827EC2AF0B3
:1072A000C80E24EC02F01200010E0501D95D0001A8
:1072B000D8A465EF39F0828AFA0E24EC02F0829AA3
:1072C000010E1D6E2C0E25EC02F0020E0501D95D9B
:1072D0000001D8A46DEF39F0828A030E0501D95D53
:1072E0000001D8A475EF39F0829A040E0501D95D2A
:1072F0000001D8A47EEF39F027EC2AF0050E050135
:10730000D95D0001D8A48CEF39F0827A949A27ECE9
:107310002AF0C80E24EC02F01200010E0501DA5D1D
:107320000001D8A49EEF39F08180FA0E24EC02F01F
:107330008190010E1D6E2C0E25EC02F0020E05014F
:10734000DA5D0001D8A4A6EF39F08180030E0501B3
:10735000DA5D0001D8A4AEEF39F08190040E05018A
:10736000DA5D0001D8A4B7EF39F027EC2AF0050E5A
:107370000501DA5D0001D8A4C5EF39F08170939062
:1073800027EC2AF0C80E24EC02F01200310E0101A5
:10739000315D0001D8A4D0EF39F0010E0101E16F99
:1073A0000001320E0101315D0001D8A4DBEF39F09C
:1073B000020E0101E16F00011200310E0101315D89
:1073C0000001D8A4E7EF39F0010E0501D86F0001E4
:1073D000320E0101315D0001D8A4F2EF39F0020E46
:1073E0000501D86F0001330E0101315D0001D8A401
:1073F000FDEF39F0030E0501D86F0001340E0101D5
:10740000315D0001D8A408EF3AF0040E0501D86FF1
:107410000001350E0101315D0001D8A413EF3AF0EF
:10742000050E0501D86F00011200310E0101315D1A
:107430000001D8A41FEF3AF0010E0501D96F000139
:10744000320E0101315D0001D8A42AEF3AF0020E9C
:107450000501D96F0001330E0101315D0001D8A48F
:1074600035EF3AF0030E0501D96F0001340E01012A
:10747000315D0001D8A440EF3AF0040E0501D96F48
:107480000001350E0101315D0001D8A44BEF3AF047
:10749000050E0501D96F00011200310E0101315DA9
:1074A0000001D8A457EF3AF0010E0501DA6F000190
:1074B000320E0101315D0001D8A462EF3AF0020EF4
:1074C0000501DA6F0001330E0101315D0001D8A41E
:1074D0006DEF3AF0030E0501DA6F0001340E010181
:1074E000315D0001D8A478EF3AF0040E0501DA6F9F
:1074F0000001350E0101315D0001D8A483EF3AF09F
:10750000050E0501DA6F00011200120012001200D0
:10751000120094928282D8960101D9A1D8860001E6
:10752000D8B69FEF3AF0170EF76E2A0EF66ED7EC2C
:1075300001F00D0EDFEC01F00A0EDFEC01F0D89641
:10754000060111ABD8860001D8B6F9EF3BF081A84F
:10755000ACEF3AF025EF40F0E86A80BA010E356EE4
:10756000E86A81B6010E3510D8B4B9EF3AF099EF58
:107570003EF0D8960501EEA9D8860001D8B6DEEF18
:107580003AF00101CE6B010ECD6F00010101CD512A
:1075900006010B5D0101CE5106010C590001D8A076
:1075A000DCEF3AF0010E24EC02F00101CD2BD8B44F
:1075B000CE2B0001D8A4E9D79394819406010951F8
:1075C0000501F35D06010A510501F4590001D8B027
:1075D000ECEF3AF090EC26F081A8F1EF3AF025EFCD
:1075E00040F0E86A80BA010E356EE86A81B6010E95
:1075F0003510D8B4FEEF3AF057EF3EF0D8960501BB
:10760000EEABD8860001D8B623EF3BF00101CE6B7C
:10761000010ECD6F00010101CD510601095D01018F
:10762000CE5106010A590001D8A021EF3BF0010E0E
:1076300024EC02F00101CD2BD8B4CE2B0001D8A44C
:10764000E9D793928192060107510501F35D060186
:1076500008510501F4590001D8B031EF3BF090EC2E
:1076600026F081A836EF3BF025EF40F0E86A80BABB
:10767000010E356EE86A81B6010E3510D8B443EFBD
:107680003BF015EF3EF0D8960501EEADD88600012F
:10769000D8B668EF3BF00101CE6B010ECD6F000153
:1076A0000101CD510601075D0101CE5106010859C6
:1076B0000001D8A066EF3BF0010E24EC02F00101BE
:1076C000CD2BD8B4CE2B0001D8A4E9D793908190CC
:1076D000060105510501F35D060106510501F45946
:1076E0000001D8B076EF3BF090EC26F081A87BEF5C
:1076F0003BF025EF40F0E86A80BA010E356EE86A8B
:1077000081B6010E3510D8B488EF3BF0D3EF3DF0D1
:10771000D8960501EEAFD8860001D8B6ADEF3BF0A4
:107720000101CE6B010ECD6F00010101CD510601AB
:10773000055D0101CE51060106590001D8A0ABEF4D
:107740003BF0010E24EC02F00101CD2BD8B4CE2B7E
:107750000001D8A4E9D7949A829A06010351050141
:10776000F35D060104510501F4590001D8B0BBEFE7
:107770003BF090EC26F081A8C0EF3BF025EF40F005
:10778000E86A80BA010E356EE86A81B6010E3510DE
:10779000D8B4CDEF3BF091EF3DF0D896060111A1A2
:1077A000D8860001D8B6F2EF3BF00101CE6B010E96
:1077B000CD6F00010101CD510601035D0101CE51E4
:1077C000060104590001D8A0F0EF3BF0010E24ECB3
:1077D00002F00101CD2BD8B4CE2B0001D8A4E9D7FB
:1077E0009498829881A8F7EF3BF025EF40F049EF9D
:1077F0003DF081A8FEEF3BF025EF40F0E86A80BA4B
:10780000010E356EE86A81B6010E3510D8B40BEF63
:107810003CF0DEEF3FF0D8960501EEA9D8860001D6
:10782000D8B630EF3CF00101CE6B010ECD6F0001F8
:107830000101CD510601035D0101CE51060104593C
:107840000001D8A02EEF3CF0010E24EC02F0010163
:10785000CD2BD8B4CE2B0001D8A4E9D79498829828
:10786000060105510501F35D060106510501F459B4
:107870000001D8B03EEF3CF090EC26F081A843EF39
:107880003CF025EF40F0E86A80BA010E356EE86AF8
:1078900081B6010E3510D8B450EF3CF09CEF3FF0AC
:1078A000D8960501EEABD8860001D8B675EF3CF04E
:1078B0000101CE6B010ECD6F00010101CD5106011A
:1078C000055D0101CE51060106590001D8A073EFF4
:1078D0003CF0010E24EC02F00101CD2BD8B4CE2BEC
:1078E0000001D8A4E9D7949A829A060107510501AC
:1078F000F35D060108510501F4590001D8B083EF8A
:107900003CF090EC26F081A888EF3CF025EF40F0A9
:10791000E86A80BA010E356EE86A81B6010E35104C
:10792000D8B495EF3CF05AEF3FF0D8960501EEAD94
:10793000D8860001D8B6BAEF3CF00101CE6B010E3B
:10794000CD6F00010101CD510601075D0101CE514E
:10795000060108590001D8A0B8EF3CF0010E24EC54
:1079600002F00101CD2BD8B4CE2B0001D8A4E9D769
:1079700093908190060109510501F35D06010A51BA
:107980000501F4590001D8B0C8EF3CF090EC26F0A6
:1079900081A8CDEF3CF025EF40F0E86A80BA010EF7
:1079A000356EE86A81B6010E3510D8B4DAEF3CF0D6
:1079B00018EF3FF0D8960501EEAFD8860001D8B693
:1079C000FFEF3CF00101CE6B010ECD6F0001010114
:1079D000CD510601095D0101CE5106010A59000190
:1079E000D8A0FDEF3CF0010E24EC02F00101CD2BFC
:1079F000D8B4CE2B0001D8A4E9D793928192060186
:107A00000B510501F35D06010C510501F45900010C
:107A1000D8B00DEF3DF090EC26F081A812EF3DF0CC
:107A200025EF40F0E86A80BA010E356EE86A81B64B
:107A3000010E3510D8B41FEF3DF0D6EF3EF0D896CA
:107A4000060111A1D8860001D8B644EF3DF001012E
:107A5000CE6B010ECD6F00010101CD5106010B5D12
:107A60000101CE5106010C590001D8A042EF3DF0B2
:107A7000010E24EC02F00101CD2BD8B4CE2B000175
:107A8000D8A4E9D79394819481A849EF3DF025EFDC
:107A900040F005012B9DD896060111B7D88600014C
:107AA000D8B655EF3DF090EC26F096EF17F0D8964B
:107AB000060111A3D8860001D8B661EF3DF096EF1C
:107AC00017F094928282D8960101D9A1D88600013C
:107AD000D8B677EF3DF0170EF76E420EF66ED7EC84
:107AE00001F00D0EDFEC01F00A0EDFEC01F0D8968C
:107AF000060111A9D8860001D8B6C5EF3EF081A8CD
:107B000084EF3DF025EF40F0010E80BAE86A356E53
:107B1000010E81B6E86A3514D8B491EF3DF025EF37
:107B200040F0D8960501EEA9D8860001D8B6B6EF88
:107B30003DF00101CE6B010ECD6F00010101CD5171
:107B40000501F55D0101CE510501F6590001D8A0EE
:107B5000B4EF3DF0010E24EC02F00101CD2BD8B4BE
:107B6000CE2B0001D8A4E9D7949882880501F7515B
:107B7000F35DF851F4590001D8B0C1EF3DF090EC3D
:107B800026F081A8C6EF3DF025EF40F0010E80BA47
:107B9000E86A356E010E81B6E86A3514D8B4D3EFC1
:107BA0003DF088EF3BF0D8960501EEABD88600019A
:107BB000D8B6F8EF3DF00101CE6B010ECD6F00019C
:107BC0000101CD510501F75D0101CE510501F859C3
:107BD0000001D8A0F6EF3DF0010E24EC02F0010107
:107BE000CD2BD8B4CE2B0001D8A4E9D7949A828AA1
:107BF0000501F951F35DFA51F4590001D8B003EFD2
:107C00003EF090EC26F081A808EF3EF025EF40F022
:107C1000010E80BAE86A356E010E81B6E86A351445
:107C2000D8B415EF3EF043EF3BF0D8960501EEAD2A
:107C3000D8860001D8B63AEF3EF00101CE6B010EB6
:107C4000CD6F00010101CD510501F95D0101CE515A
:107C50000501FA590001D8A038EF3EF0010E24ECDE
:107C600002F00101CD2BD8B4CE2B0001D8A4E9D766
:107C7000939081800501FB51F35DFC51F4590001A3
:107C8000D8B045EF3EF090EC26F081A84AEF3EF0E8
:107C900025EF40F0010E80BAE86A356E010E81B61C
:107CA000E86A3514D8B457EF3EF0FEEF3AF0D896B4
:107CB0000501EEAFD8860001D8B67CEF3EF0010199
:107CC000CE6B010ECD6F00010101CD510501FB5DB1
:107CD0000101CE510501FC590001D8A07AEF3EF018
:107CE000010E24EC02F00101CD2BD8B4CE2B000103
:107CF000D8A4E9D7939281820501FD51F35DFE512D
:107D0000F4590001D8B087EF3EF090EC26F081A83E
:107D10008CEF3EF025EF40F0010E80BAE86A356E38
:107D2000010E81B6E86A3514D8B499EF3EF0B9EF88
:107D30003AF0D896060111A1D8860001D8B6BEEF58
:107D40003EF00101CE6B010ECD6F00010101CD515E
:107D50000501FD5D0101CE510501FE590001D8A0CC
:107D6000BCEF3EF0010E24EC02F00101CD2BD8B4A3
:107D7000CE2B0001D8A4E9D79394818481A8C3EFC6
:107D80003EF025EF40F008EF40F081A8CAEF3EF04A
:107D900025EF40F0010E80BAE86A356E010E81B61B
:107DA000E86A3514D8B4D6EF3EF049D6D896050126
:107DB000EEA9D8860001D8B6FBEF3EF00101CE6BEC
:107DC000010ECD6F00010101CD510501FD5D0101E5
:107DD000CE510501FE590001D8A0F9EF3EF0010E89
:107DE00024EC02F00101CD2BD8B4CE2B0001D8A495
:107DF000E9D7939481840501FB51F35DFC51F4595B
:107E00000001D8B006EF3FF090EC26F081A80BEF10
:107E10003FF025EF40F0010E80BAE86A356E010EA2
:107E200081B6E86A3514D8B418EF3FF0DAEF3CF0C9
:107E3000D8960501EEABD8860001D8B63DEF3FF0ED
:107E40000101CE6B010ECD6F00010101CD51050185
:107E5000FB5D0101CE510501FC590001D8A03BEFAB
:107E60003FF0010E24EC02F00101CD2BD8B4CE2B53
:107E70000001D8A4E9D7939281820501F951F35DFD
:107E8000FA51F4590001D8B048EF3FF090EC26F0D9
:107E900081A84DEF3FF025EF40F0010E80BAE86A6F
:107EA000356E010E81B6E86A3514D8B45AEF3FF04A
:107EB00095EF3CF0D8960501EEADD8860001D8B616
:107EC0007FEF3FF00101CE6B010ECD6F000101018C
:107ED000CD510501F95D0101CE510501FA590001AD
:107EE000D8A07DEF3FF0010E24EC02F00101CD2B74
:107EF000D8B4CE2B0001D8A4E9D793908180050196
:107F0000F751F35DF851F4590001D8B08AEF3FF012
:107F100090EC26F081A88FEF3FF025EF40F0010EA6
:107F200080BAE86A356E010E81B6E86A3514D8B4B5
:107F30009CEF3FF050EF3CF0D8960501EEAFD886AD
:107F40000001D8B6C1EF3FF00101CE6B010ECD6F3D
:107F500000010101CD510501F75D0101CE5105017F
:107F6000F8590001D8A0BFEF3FF0010E24EC02F059
:107F70000101CD2BD8B4CE2B0001D8A4E9D7949A17
:107F8000828A0501F551F35DF651F4590001D8B02C
:107F9000CCEF3FF090EC26F081A8D1EF3FF025EF39
:107FA00040F0010E80BAE86A356E010E81B6E86ACB
:107FB0003514D8B4DEEF3FF00BEF3CF0D896060155
:107FC00011A1D8860001D8B603EF40F00101CE6BB5
:107FD000010ECD6F00010101CD510501F55D0101DB
:107FE000CE510501F6590001D8A001EF40F0010E75
:107FF00024EC02F00101CD2BD8B4CE2B0001D8A483
:10800000E9D79498828881A808EF40F025EF40F0E6
:1080100005012B8DD896060111B7D8860001D8B678
:1080200014EF40F090EC26F096EF17F005012B9D31
:10803000000196EF17F005012B8D000181A823EFB9
:1080400040F025EF40F096EF17F081EC2BF096EF23
:1080500017F0170EF76E580EF66E01EE31F001ECC8
:1080600003F0D8A437EF40F0010E01016B6F00015F
:10807000170EF76E600EF66E01EE31F001EC03F0B4
:10808000D8A451EF40F001016B6B04EEA5F0170E80
:10809000F76E680EF66ED9EC02F0EF6A0001E4ECC0
:1080A0001DF0170EF76E7E0EF66E01EE31F001EC4C
:1080B00003F0D8A46BEF40F0020E01016B6F04EEE9
:1080C000A5F0170EF76E840EF66ED9EC02F0EF6A8B
:1080D0000001E4EC1DF01200170EF76E980EF66E1C
:1080E00001EE31F001EC03F0D8A47FEF40F006017F
:1080F0001187010E0101686F00018FEF40F006014A
:1081000011970101686B04EEA5F0170EF76E9C0E37
:10811000F66ED9EC02F0EF6A0001E4EC1DF01200FB
:10812000170EF76EAC0EF66E01EE31F001EC03F0B7
:10813000D8A4A0EF40F0060111970101686B696BAC
:108140000001170EF76EB20EF66E01EE31F001EC83
:1081500003F0D8A4B3EF40F006011187010E01012E
:10816000686F010E696F0001120005EED1F011EE8B
:1081700031F0060EE6CFEEFFE82EFCD7EF6A04EEF4
:10818000A5F0170EF76EBA0EF66ED9EC02F015EEEA
:10819000D1F0060EE75204E0E6CFEEFFE82EFAD764
:1081A000EF6AE4EC1DF0120005EE93F015EED1F04D
:1081B000060EE75204E0E6CFEEFFE82EFAD7EF6AAC
:1081C00089EC2CF0120004EEA5F0170EF76ECC0E21
:1081D000F66ED9EC02F011EE31F0360EE75204E003
:1081E000E6CFEEFFE82EFAD7EF6AE4EC1DF001EEE1
:1081F00031F084EC00F00501E06F21C0E1F50001F1
:10820000120004EEA5F0170EF76EE20EF66ED9EC32
:1082100002F011EE31F0360EE75204E0E6CFEEFF49
:10822000E82EFAD7EF6AE4EC1DF001EE31F084ECB1
:1082300000F00501E26F21C0E3F5000112000AEC35
:1082400039F004EEA5F0170EF76EFA0EF66ED9ECC3
:1082500002F0020E016E0501ED51CCEC00F0EF6A68
:108260000001E4EC1DF0120004EEA5F0180EF76E0C
:10827000120EF66ED9EC02F011EE31F0360EE75226
:1082800004E0E6CFEEFFE82EFAD72E0EEE6EEF6A90
:10829000E4EC1DF001EE31F084EC00F00501ED6F2F
:1082A0000001120004EEA5F0180EF76E2E0EF66E09
:1082B000D9EC02F011EE31F0360EE75204E0E6CFD1
:1082C000EEFFE82EFAD7200EEE6E6D0EEE6E730EF8
:1082D000EE6E2E0EEE6EEF6AE4EC1DF001EE31F064
:1082E00084EC00F00501F56F21C0F6F500011200E5
:1082F00004EEA5F0180EF76E440EF66ED9EC02F0FF
:1083000011EE31F0360EE75204E0E6CFEEFFE82E34
:10831000FAD7200EEE6E6D0EEE6E730EEE6E2E0E12
:10832000EE6EEF6AE4EC1DF001EE31F084EC00F04B
:108330000501F76F21C0F8F50001120004EEA5F069
:10834000180EF76E5A0EF66ED9EC02F011EE31F0FF
:10835000360EE75204E0E6CFEEFFE82EFAD7200E05
:10836000EE6E6D0EEE6E730EEE6E2E0EEE6EEF6A0C
:10837000E4EC1DF001EE31F084EC00F00501F96F42
:1083800021C0FAF50001120004EEA5F0180EF76EF8
:10839000700EF66ED9EC02F011EE31F0360EE752A7
:1083A00004E0E6CFEEFFE82EFAD7200EEE6E6D0E5B
:1083B000EE6E730EEE6E2E0EEE6EEF6AE4EC1DF0B6
:1083C00001EE31F084EC00F00501FB6F21C0FCF5FB
:1083D0000001120004EEA5F0180EF76E860EF66E80
:1083E000D9EC02F011EE31F0360EE75204E0E6CFA0
:1083F000EEFFE82EFAD7200EEE6E6D0EEE6E730EC7
:10840000EE6E2E0EEE6EEF6AE4EC1DF001EE31F032
:1084100084EC00F00501FD6F21C0FEF500011200A3
:1084200004EEA5F0180EF76E9C0EF66ED9EC02F075
:1084300011EE31F0360EE75204E0E6CFEEFFE82E03
:10844000FAD7200EEE6E6D0EEE6E730EEE6E2E0EE1
:10845000EE6EEF6AE4EC1DF001EE31F084EC00F01A
:108460000601036F21C004F60001120004EEA5F01E
:10847000180EF76EB00EF66ED9EC02F011EE31F078
:10848000360EE75204E0E6CFEEFFE82EFAD7200ED4
:10849000EE6E6D0EEE6E730EEE6E2E0EEE6EEF6ADB
:1084A000E4EC1DF001EE31F084EC00F00601056F04
:1084B00021C006F60001120004EEA5F0180EF76EBA
:1084C000C40EF66ED9EC02F011EE31F0360EE75222
:1084D00004E0E6CFEEFFE82EFAD7200EEE6E6D0E2A
:1084E000EE6E730EEE6E2E0EEE6EEF6AE4EC1DF085
:1084F00001EE31F084EC00F00601076F21C008F6B0
:108500000001120004EEA5F0180EF76ED80EF66EFC
:10851000D9EC02F011EE31F0360EE75204E0E6CF6E
:10852000EEFFE82EFAD7200EEE6E6D0EEE6E730E95
:10853000EE6E2E0EEE6EEF6AE4EC1DF001EE31F001
:1085400084EC00F00601096F21C00AF60001120058
:1085500004EEA5F0180EF76EEC0EF66ED9EC02F0F4
:1085600011EE31F0360EE75204E0E6CFEEFFE82ED2
:10857000FAD7200EEE6E6D0EEE6E730EEE6E2E0EB0
:10858000EE6EEF6AE4EC1DF001EE31F084EC00F0E9
:1085900006010B6F21C00CF600011200310E010123
:1085A000315D0001D8A4DCEF42F00501EE8901EE57
:1085B000A0F0310EEE6EEF6A0001320E0101315D66
:1085C0000001D8A4EBEF42F00501EE8B01EEA0F024
:1085D000320EEE6EEF6A0001330E0101315D0001D3
:1085E000D8A4FAEF42F00501EE8D01EEA0F0330EB3
:1085F000EE6EEF6A0001340E0101315D0001D8A476
:1086000009EF43F00501EE8F01EEA0F0340EEE6E9F
:10861000EF6A0001350E0101315D0001D8A418EFA9
:1086200043F00601118101EEA0F0350EEE6EEF6A07
:10863000000104EEA5F0190EF76E000EF66ED9ECEF
:1086400002F011EEA0F0140EE75204E0E6CFEEFFC8
:10865000E82EFAD7190EF76E080EF66ED9EC02F076
:10866000EF6AE4EC1DF01200310E0101315D0001F2
:10867000D8A442EF43F00501EE9901EEA0F0310ECF
:10868000EE6EEF6A0001320E0101315D0001D8A4E7
:1086900051EF43F00501EE9B01EEA0F0320EEE6EBD
:1086A000EF6A0001330E0101315D0001D8A460EFD3
:1086B00043F00501EE9D01EEA0F0330EEE6EEF6A81
:1086C0000001340E0101315D0001D8A46FEF43F0C9
:1086D0000501EE9F01EEA0F0340EEE6EEF6A000190
:1086E000350E0101315D0001D8A47EEF43F0060193
:1086F000119101EEA0F0350EEE6EEF6A000104EE6E
:10870000A5F0190EF76E120EF66ED9EC02F011EE0E
:10871000A0F0140EE75204E0E6CFEEFFE82EFAD701
:10872000190EF76E1A0EF66ED9EC02F0EF6AE4EC51
:108730001DF01200190EF76E240EF66E01EE31F0E8
:1087400001EC03F0D8A4A6EF43F08288190EF76E6F
:10875000280EF66E01EE31F001EC03F0D8A4B2EF72
:1087600043F0829882A8C0EF43F004EEA5F0190E02
:10877000F76E2C0EF66ED9EC02F0EF6AE4EC1DF009
:1087800082B8CEEF43F004EEA5F0190EF76E3E0E60
:10879000F66ED9EC02F0EF6AE4EC1DF01200190E4F
:1087A000F76E500EF66E01EE31F001EC03F0D8A436
:1087B000DBEF43F0828A190EF76E540EF66E01EE6F
:1087C00031F001EC03F0D8A4E7EF43F0829A82AADB
:1087D000F5EF43F004EEA5F0190EF76E580EF66EA5
:1087E000D9EC02F0EF6AE4EC1DF082BA03EF44F03A
:1087F00004EEA5F0190EF76E6A0EF66ED9EC02F0D3
:10880000EF6AE4EC1DF01200190EF76E7C0EF66EA6
:1088100001EE31F001EC03F0D8A410EF44F08180B8
:10882000190EF76E800EF66E01EE31F001EC03F0DA
:10883000D8A41CEF44F0819081A02AEF44F004EE0C
:10884000A5F0190EF76E840EF66ED9EC02F0EF6A01
:10885000E4EC1DF081B038EF44F004EEA5F0190E01
:10886000F76E960EF66ED9EC02F0EF6AE4EC1DF0AE
:108870001200190EF76EA80EF66E01EE31F001EC43
:1088800003F0D8A445EF44F08182190EF76EAC0EC8
:10889000F66E01EE31F001EC03F0D8A451EF44F094
:1088A000819281A25FEF44F004EEA5F0190EF76EFD
:1088B000B00EF66ED9EC02F0EF6AE4EC1DF081B276
:1088C0006DEF44F004EEA5F0190EF76EC20EF66ED1
:1088D000D9EC02F0EF6AE4EC1DF01200190EF76E0D
:1088E000D40EF66E01EE31F001EC03F0D8A47AEF6D
:1088F00044F08184190EF76ED80EF66E01EE31F059
:1089000001EC03F0D8A486EF44F0819481A494EFA5
:1089100044F004EEA5F0190EF76EDC0EF66ED9ECFD
:1089200002F0EF6AE4EC1DF081B4A2EF44F004EE33
:10893000A5F0190EF76EEE0EF66ED9EC02F0EF6AA6
:10894000E4EC1DF012001A0EF76E000EF66E01EE4A
:1089500031F001EC03F0D8A4B0EF44F00601138F1E
:1089600000011A0EF76E040EF66E01EE31F001EC06
:1089700003F0D8A4BEEF44F00601139F0001D8967F
:10898000060113AFD8860001D8B6D2EF44F004EE4A
:10899000A5F01A0EF76E080EF66ED9EC02F0EF6A2B
:1089A000E4EC1DF0D896060113BFD8860001D8B6B6
:1089B000E5EF44F004EEA5F01A0EF76E180EF66E11
:1089C000D9EC02F0EF6AE4EC1DF00601118D000114
:1089D00012001A0EF76E2A0EF66E01EE31F001EC5F
:1089E00003F0D8A4F6EF44F00601148100011A0E3A
:1089F000F76E2E0EF66E01EE31F001EC03F0D8A406
:108A000004EF45F0060114910001D896060114A167
:108A1000D8860001D8B618EF45F004EEA5F01A0E7E
:108A2000F76E320EF66ED9EC02F0EF6AE4EC1DF050
:108A3000D896060114B1D8860001D8B62BEF45F0C0
:108A400004EEA5F01A0EF76E420EF66ED9EC02F0A7
:108A5000EF6AE4EC1DF00601118D000112001A0E00
:108A6000F76E540EF66E01EE31F001EC03F0D8A46F
:108A70003CEF45F00601148300011A0EF76E580E04
:108A8000F66E01EE31F001EC03F0D8A44AEF45F0A8
:108A9000060114930001D896060114A3D88600019C
:108AA000D8B65EEF45F004EEA5F01A0EF76E5C0E38
:108AB000F66ED9EC02F0EF6AE4EC1DF0D8960601F0
:108AC00014B3D8860001D8B671EF45F004EEA5F0D6
:108AD0001A0EF76E6C0EF66ED9EC02F0EF6AE4EC4B
:108AE0001DF00601118D00011200310E0101315DF2
:108AF0000001D8A481EF45F08288FA0E24EC02F040
:108B00008298320E0101315D0001D8A48DEF45F04D
:108B1000828AFA0E24EC02F0829A330E0101315D52
:108B20000001D8A499EF45F08180FA0E24EC02F000
:108B30008190340E0101315D0001D8A4A5EF45F00C
:108B40008182FA0E24EC02F08192350E0101315D32
:108B50000001D8A4B1EF45F08184FA0E24EC02F0B4
:108B600081940601118D0001120004EEA5F01A0E89
:108B7000F76E7E0EF66ED9EC02F0EF6AE4EC1DF0B3
:108B8000010E0501ED6F010EEB6FF66B010EF56F37
:108B9000F86B640EF76FFA6B640EF96FFC6B640E82
:108BA000FB6FFE6B640EFD6F0601006B640E05012A
:108BB000FF6F0601026B640E016F046B010E036F01
:108BC000066B640E056F086B640E076F0A6B640E0C
:108BD000096F0C6B640E0B6F0E6B640E0D6F106BD8
:108BE000640E0F6F1189118B05012B85140E916F87
:108BF000786BCD0E7C6FCC0E7B6F4C0E7A6F7C0E3B
:108C0000796F0601119505014B6B4A6B496B486BF7
:108C10004F6B4E6B4D6B4C6B536B526B516B506B80
:108C2000576B566B556B546B010169530001D8A407
:108C30001CEF46F093EC4DF0020E01016B6F686B78
:108C4000060111970501266B5B6B5A6B596B586BCC
:108C50005F6B5E6B5D6B5C6B636B626B616B606BC0
:108C6000676B666B656B646B6B6B6A6B700E696FC1
:108C7000830E686F6F6B6E6B700E6D6F830E6C6F13
:108C8000736B726B700E716F830E706F776B766B98
:108C9000700E756F830E746F0401A46B01016C6B11
:108CA0000501F46BFA0EF36F020E0101E16F010E84
:108CB0000501D86F010ED96F010EDA6FDB6BDC6B2B
:108CC000DD6BDE6B00011200010E0501DF6FAA6A89
:108CD000A96ADF51FEEC01F00A0E24EC02F0AA6A48
:108CE000020EA96EE051FEEC01F0E151FEEC01F044
:108CF0000A0E24EC02F0AA6A040EA96EE251FEEC00
:108D000001F0E351FEEC01F00A0E24EC02F0AA6A35
:108D1000060EA96EED51FEEC01F00A0E24EC02F0F5
:108D2000AA6A0A0EA96E000EFEEC01F0AA6A140EE1
:108D3000A96EF551FEEC01F0F651FEEC01F00A0EC1
:108D400024EC02F0AA6A160EA96EF751FEEC01F0AF
:108D5000F851FEEC01F00A0E24EC02F0AA6A180E9B
:108D6000A96EF951FEEC01F0FA51FEEC01F00A0E89
:108D700024EC02F0AA6A1A0EA96EFB51FEEC01F077
:108D8000FC51FEEC01F00A0E24EC02F0AA6A1C0E63
:108D9000A96EFD51FEEC01F0FE51FEEC01F00A0E51
:108DA00024EC02F0AA6A1E0EA96EFF51FEEC01F03F
:108DB00006010051FEEC01F00A0E24EC02F0AA6A52
:108DC000200EA96E0151FEEC01F00251FEEC01F003
:108DD0000A0E24EC02F0AA6A280EA96E0351FEECDA
:108DE00001F00451FEEC01F00A0E24EC02F0AA6A34
:108DF0002A0EA96E0551FEEC01F00651FEEC01F0C1
:108E00000A0E24EC02F0AA6A2C0EA96E0751FEECA1
:108E100001F00851FEEC01F00A0E24EC02F0AA6AFF
:108E20002E0EA96E0951FEEC01F00A51FEEC01F084
:108E30000A0E24EC02F0AA6A300EA96E0B51FEEC69
:108E400001F00C51FEEC01F00A0E24EC02F0AA6ACB
:108E5000320EA96E0D51FEEC01F00E51FEEC01F048
:108E60000A0E24EC02F0AA6A340EA96E0F51FEEC31
:108E700001F01051FEEC01F00A0E24EC02F0AA6A97
:108E80003C0EA96EE86A11B9010EFEEC01F00A0E63
:108E900024EC02F0AA6A3E0EA96EE86A11BB010E2C
:108EA000FEEC01F00A0E24EC02F0AA6A400EA96E54
:108EB0000401A451FEEC01F00A0E24EC02F0AA6AAF
:108EC000410EA96E05EED1F0EE5003E0FEEC01F08C
:108ED000FBD70A0E24EC02F001EECAF015EED1F039
:108EE000010EF36E010EE1EC02F0EF6AAA6A410E88
:108EF000A96E01EECAF0EE5003E0FEEC01F0FBD7E4
:108F00000A0E24EC02F001EECAF015EED1F0020ECA
:108F1000F36E010EE1EC02F0EF6AAA6A420EA96E4E
:108F200001EECAF0EE5003E0FEEC01F0FBD70A0EB2
:108F300024EC02F001EECAF015EED1F0030EF36E50
:108F4000010EE1EC02F0EF6AAA6A430EA96E01EE8F
:108F5000CAF0EE5003E0FEEC01F0FBD70A0E24EC61
:108F600002F001EECAF015EED1F0040EF36E010E20
:108F7000E1EC02F0EF6AAA6A440EA96E01EECAF0B3
:108F8000EE5003E0FEEC01F0FBD70A0E24EC02F0F9
:108F900001EECAF015EED1F0050EF36E010EE1EC14
:108FA00002F0EF6AAA6A450EA96E01EECAF0EE5011
:108FB00003E0FEEC01F0FBD70A0E24EC02F001EE18
:108FC000CAF015EED1F0060EF36E010EE1EC02F0E0
:108FD000EF6AAA6A460EA96E01EECAF0EE5003E0EF
:108FE000FEEC01F0FBD70A0E24EC02F0AA6A500E48
:108FF000A96EE86A0501EEB9010EFEEC01F00A0E59
:1090000024EC02F0AA6A510EA96EE86AEEBB010ECA
:10901000FEEC01F00A0E24EC02F0AA6A520EA96ED0
:10902000E86AEEBD010EFEEC01F00A0E24EC02F03F
:10903000AA6A530EA96EE86AEEBF010EFEEC01F0BB
:109040000A0E24EC02F0AA6A540EA96EE86A060120
:1090500011B1010EFEEC01F00A0E24EC02F0AA6A36
:10906000550EA96E05019151FEEC01F00A0E24EC9B
:1090700002F0AA6A560EA96E7851FEEC01F00A0EB3
:1090800024EC02F0AA6A570EA96E7951FEEC01F0A9
:109090007A51FEEC01F07B51FEEC01F07C51FEECCC
:1090A00001F00A0E24EC02F0AA6A5B0EA96EE86ACF
:1090B000060111B7010EFEEC01F00A0E24EC02F0DD
:1090C000AA6A5C0EA96E05014851FEEC01F04951F7
:1090D000FEEC01F04A51FEEC01F04B51FEEC01F0C8
:1090E0000A0E24EC02F0AA6A600EA96E4C51FEEC46
:1090F00001F04D51FEEC01F04E51FEEC01F04F51EC
:10910000FEEC01F00A0E24EC02F0AA6A640EA96ECD
:109110005051FEEC01F05151FEEC01F05251FEECC9
:1091200001F05351FEEC01F00A0E24EC02F0AA6AA1
:10913000680EA96E5451FEEC01F05551FEEC01F0A1
:109140005651FEEC01F05751FEEC01F00A0E24ECF2
:1091500002F0AA6A6C0EA96E01016851FEEC01F0E2
:109160000A0E24EC02F0AA6A6D0EA96E6951FEEC9B
:1091700001F00A0E24EC02F0AA6A6E0EA96E6B5181
:10918000FEEC01F00A0E24EC02F0AA6A6F0EA96E42
:1091900005015851FEEC01F05951FEEC01F05A5115
:1091A000FEEC01F05B51FEEC01F00A0E24EC02F043
:1091B000AA6A730EA96E5C51FEEC01F05D51FEECE3
:1091C00001F05E51FEEC01F05F51FEEC01F00A0E81
:1091D00024EC02F0AA6A770EA96E6051FEEC01F051
:1091E0006151FEEC01F06251FEEC01F06351FEECC6
:1091F00001F00A0E24EC02F0AA6A7B0EA96E6451FB
:10920000FEEC01F06551FEEC01F06651FEEC01F060
:109210006751FEEC01F00A0E24EC02F0AA6A7F0E00
:10922000A96E6851FEEC01F06951FEEC01F06A5143
:10923000FEEC01F06B51FEEC01F00A0E24EC02F0A2
:10924000AA6A830EA96E6C51FEEC01F06D51FEEC22
:1092500001F06E51FEEC01F06F51FEEC01F00A0ED0
:1092600024EC02F0AA6A870EA96E7051FEEC01F0A0
:109270007151FEEC01F07251FEEC01F07351FEEC05
:1092800001F00A0E24EC02F0AA6A8B0EA96E74514A
:10929000FEEC01F07551FEEC01F07651FEEC01F0B0
:1092A0007751FEEC01F00A0E24EC02F0AA6A8F0E50
:1092B000A96E01016C51FEEC01F00A0E24EC02F0E3
:1092C000AA6A900EA96E05012651FEEC01F00A0E65
:1092D00024EC02F0AA6A910EA96EF351FEEC01F0A3
:1092E000F451FEEC01F00A0E24EC02F0AA6A930E8F
:1092F000A96E0101E151FEEC01F00A0E24EC02F02E
:10930000AA6A940EA96E0501D851FEEC01F00A0E6E
:1093100024EC02F0AA6A950EA96ED951FEEC01F078
:109320000A0E24EC02F0AA6A960EA96EDA51FEEC3F
:1093300001F00A0E24EC02F0AA6A970EA96EDB5126
:10934000FEEC01F00A0E24EC02F0AA6A980EA96E57
:10935000DC51FEEC01F00A0E24EC02F0AA6A990E30
:10936000A96EDD51FEEC01F00A0E24EC02F0AA6AAF
:109370009A0EA96EDE51FEEC01F00A0E24EC02F00A
:10938000AA6A9B0EA96EE86A2BB5010EFEEC01F0ED
:109390000A0E24EC02F004EEA5F01A0EF76EA60EEB
:1093A000F66ED9EC02F0EF6A0001E4EC1DF0120059
:1093B000000EF5EC01F00501DF6F020EF5EC01F097
:1093C000E06FF7EC01F0E16F040EF5EC01F0E26FF5
:1093D000F7EC01F0E36F060EF5EC01F0ED6F0A0E0D
:1093E000F5EC01F0EB6FEB29EC6F140EF5EC01F0EE
:1093F000F56FF7EC01F0F66F160EF5EC01F0F76F74
:10940000F7EC01F0F86F180EF5EC01F0F96FF7ECDE
:1094100001F0FA6F1A0EF5EC01F0FB6FF7EC01F0BA
:10942000FC6F1C0EF5EC01F0FD6FF7EC01F0FE6F28
:109430001E0EF5EC01F0FF6FF7EC01F00601006F76
:10944000200EF5EC01F0016FF7EC01F0026F280E31
:10945000F5EC01F0036FF7EC01F0046F2A0EF5EC68
:1094600001F0056FF7EC01F0066F2C0EF5EC01F042
:10947000076FF7EC01F0086F2E0EF5EC01F0096FA5
:10948000F7EC01F00A6F300EF5EC01F00B6FF7EC22
:1094900001F00C6F320EF5EC01F00D6FF7EC01F0FE
:1094A0000E6F340EF5EC01F00F6FF7EC01F0106F5A
:1094B0003C0EF5EC01F01189E8A011993E0EF5EC97
:1094C00001F0118BE8A0119B400EF5EC01F00401B6
:1094D000A46F500EF5EC01F00501EE89E8A0EE99BD
:1094E000510EF5EC01F0EE8BE8A0EE9B520EF5EC80
:1094F00001F0EE8DE8A0EE9D530EF5EC01F0EE8F3D
:10950000E8A0EE9F540EF5EC01F006011181E8A0F1
:109510001191550EF5EC01F00501916F560EF5EC29
:1095200001F0786F570EF5EC01F0796FF7EC01F070
:109530007A6FF7EC01F07B6FF7EC01F07C6F5B0E5C
:10954000F5EC01F006011187E8A011975C0EF5EC2F
:1095500001F00501486FF7EC01F0496FF7EC01F0FD
:109560004A6FF7EC01F04B6F600EF5EC01F04C6FB9
:10957000F7EC01F04D6FF7EC01F04E6FF7EC01F0F6
:109580004F6F640EF5EC01F0506FF7EC01F0516F86
:10959000F7EC01F0526FF7EC01F0536F680EF5EC49
:1095A00001F0546FF7EC01F0556FF7EC01F0566FD6
:1095B000F7EC01F0576F6C0EF5EC01F00101686FEC
:1095C0006D0EF5EC01F0696F6E0EF5EC01F06B6F4E
:1095D0006F0EF5EC01F00501586FF7EC01F0596FD3
:1095E000F7EC01F05A6FF7EC01F05B6F730EF5ECDE
:1095F00001F05C6FF7EC01F05D6FF7EC01F05E6F6E
:10960000F7EC01F05F6F770EF5EC01F0606FF7ECAF
:1096100001F0616FF7EC01F0626FF7EC01F0636F3E
:109620007B0EF5EC01F0646FF7EC01F0656FF7EC81
:1096300001F0666FF7EC01F0676F7F0EF5EC01F05B
:10964000686FF7EC01F0696FF7EC01F06A6FF7EC07
:1096500001F06B6F830EF5EC01F06C6FF7EC01F02D
:109660006D6FF7EC01F06E6FF7EC01F06F6F870E26
:10967000F5EC01F0706FF7EC01F0716FF7EC01F0B1
:10968000726FF7EC01F0736F8B0EF5EC01F0746FF5
:10969000F7EC01F0756FF7EC01F0766FF7EC01F085
:1096A000776F8F0EF5EC01F001016C6F900EF5EC09
:1096B00001F00501266F910EF5EC01F0F36FF7EC68
:1096C00001F0F46F930EF5EC01F00101E16F940EDF
:1096D000F5EC01F00501D86F950EF5EC01F0D96FAE
:1096E000960EF5EC01F0DA6F970EF5EC01F0DB6FFA
:1096F000980EF5EC01F0DC6F990EF5EC01F0DD6FE2
:109700009A0EF5EC01F0DE6F9B0EF5EC01F02B8567
:10971000E8A02B95130EF65D0001D8A09EEF4BF04C
:10972000D8A49AEF4BF0890E0501F55D0001D8A091
:109730009EEF4BF00501F66B320EF56F0001010153
:109740006B530001D8A4A7EF4BF093EC4DF001014F
:109750006B530001D8A4B8EF4BF004EEA5F01A0E3D
:10976000F76ECC0EF66ED9EC02F0EF6AE4EC1DF069
:10977000020E01016B5D0001D8A4D9EF4BF004EE9D
:10978000A5F01A0EF76EF40EF66ED9EC02F01B0E71
:10979000F76E060EF66ED9EC02F0020E016E0501B0
:1097A000ED51CCEC00F0290EEE6EEF6A0001E4EC16
:1097B0001DF0120004EEA5F01B0EF76E100EF66EF3
:1097C000D9EC02F0EF6AE4EC1DF004EEA5F01B0EFC
:1097D000F76E640EF66ED9EC02F0EF6AE4EC1DF061
:1097E00004EEA5F01B0EF76EB60EF66ED9EC02F085
:1097F000EF6AE4EC1DF004EEA5F01C0EF76E080E07
:10980000F66ED9EC02F0EF6AE4EC1DF004EEA5F080
:109810001C0EF76E500EF66ED9EC02F0EF6AE4EC17
:109820001DF004EEA5F01C0EF76E980EF66ED9EC46
:1098300002F0EF6AE4EC1DF004EEA5F01C0EF76EEA
:10984000D60EF66ED9EC02F0EF6AE4EC1DF004EEF1
:10985000A5F01D0EF76E140EF66ED9EC02F0EF6A4D
:10986000E4EC1DF004EEA5F01D0EF76E3C0EF66E56
:10987000D9EC02F0EF6AE4EC1DF004EEA5F01D0E49
:10988000F76E660EF66ED9EC02F0EF6AE4EC1DF0AE
:1098900004EEA5F01D0EF76EBA0EF66ED9EC02F0CE
:1098A000EF6AE4EC1DF004EEA5F01D0EF76EEA0E73
:1098B000F66ED9EC02F0EF6AE4EC1DF004EEA5F0D0
:1098C0001E0EF76E1E0EF66ED9EC02F0EF6AE4EC97
:1098D0001DF004EEA5F01E0EF76E540EF66ED9ECD8
:1098E00002F0EF6AE4EC1DF004EEA5F01E0EF76E38
:1098F000880EF66ED9EC02F0EF6AE4EC1DF004EE8F
:10990000A5F01E0EF76ED00EF66ED9EC02F0EF6ADF
:10991000E4EC1DF004EEA5F01E0EF76EF40EF66EEC
:10992000D9EC02F0EF6AE4EC1DF004EEA5F01F0E96
:10993000F76E1C0EF66ED9EC02F0EF6AE4EC1DF047
:1099400004EEA5F01F0EF76E440EF66ED9EC02F091
:10995000EF6AE4EC1DF004EEA5F01F0EF76E960E14
:10996000F66ED9EC02F0EF6AE4EC1DF004EEA5F01F
:109970001F0EF76EEA0EF66ED9EC02F0EF6AE4EC19
:109980001DF004EEA5F0200EF76E4A0EF66ED9EC2F
:1099900002F0EF6AE4EC1DF004EEA5F0200EF76E85
:1099A000920EF66ED9EC02F0EF6AE4EC1DF004EED4
:1099B000A5F0200EF76EDC0EF66ED9EC02F0EF6A21
:1099C000E4EC1DF004EEA5F0210EF76E0C0EF66E21
:1099D000D9EC02F0EF6AE4EC1DF004EEA5F0210EE4
:1099E000F76E600EF66ED9EC02F0EF6AE4EC1DF053
:1099F00004EEA5F0210EF76EB20EF66ED9EC02F071
:109A0000EF6AE4EC1DF004EEA5F0220EF76E080EEE
:109A1000F66ED9EC02F0EF6AE4EC1DF004EEA5F06E
:109A2000220EF76E4C0EF66ED9EC02F0EF6AE4EC03
:109A30001DF004EEA5F0220EF76E920EF66ED9EC34
:109A400002F0EF6AE4EC1DF004EEA5F0220EF76ED2
:109A5000E60EF66ED9EC02F0EF6AE4EC1DF004EECF
:109A6000A5F0230EF76E320EF66ED9EC02F0EF6A17
:109A7000E4EC1DF004EEA5F0230EF76E700EF66E0A
:109A8000D9EC02F0EF6AE4EC1DF004EEA5F0230E31
:109A9000F76EB80EF66ED9EC02F0EF6AE4EC1DF04A
:109AA00004EEA5F0230EF76EFA0EF66ED9EC02F076
:109AB000EF6AE4EC1DF004EEA5F0240EF76E4E0EF6
:109AC000F66ED9EC02F0EF6AE4EC1DF004EEA5F0BE
:109AD000240EF76E800EF66ED9EC02F0EF6AE4EC1D
:109AE0001DF004EEA5F0240EF76EB20EF66ED9EC62
:109AF00002F0EF6AE4EC1DF004EEA5F0250EF76E1F
:109B0000060EF66ED9EC02F0EF6AE4EC1DF004EEFE
:109B1000A5F0250EF76E460EF66ED9EC02F0EF6A50
:109B2000E4EC1DF0120004EEA5F0250EF76E9A0E7F
:109B3000F66ED9EC02F0EF6AE4EC1DF001EE6DF088
:109B4000020E016E0501DF51CCEC00F0EF6A04EE6D
:109B5000A5F0250EF76EC20EF66ED9EC02F011EEEE
:109B60006DF0320EE75204E0E6CFEEFFE82EFAD7B2
:109B7000EF6A0001E4EC1DF001EE6DF015EEE4F08B
:109B8000060EE75204E0E6CFEEFFE82EFAD7EF6AC2
:109B900004EEA5F0250EF76ED20EF66ED9EC02F0AB
:109BA00011EE6DF0320EE75204E0E6CFEEFFE82E44
:109BB000FAD7EF6AE4EC1DF001EE6DF0020E016ED3
:109BC000086AE1C521F0E0C520F0CFEC00F0EF6AB3
:109BD00004EEA5F0250EF76EE20EF66ED9EC02F05B
:109BE00011EE6DF0320EE75204E0E6CFEEFFE82E04
:109BF000FAD7EF6AE4EC1DF001EE6DF0020E016E93
:109C0000086AE3C521F0E2C520F0CFEC00F0EF6A6E
:109C100004EEA5F0250EF76EF20EF66ED9EC02F00A
:109C200011EE6DF0320EE75204E0E6CFEEFFE82EC3
:109C3000FAD7EF6AE4EC1DF001EE6DF0020E016E52
:109C40000501ED51CCEC00F0EF6A04EEA5F0260E14
:109C5000F76E020EF66ED9EC02F011EE6DF0320ED8
:109C6000E75204E0E6CFEEFFE82EFAD7EF6A0001F4
:109C7000E4EC1DF001EE6DF0020E016E086AF6C50F
:109C800021F0F5C520F0CFEC00F0EF6A04EEA5F06E
:109C9000260EF76E120EF66ED9EC02F011EE6DF094
:109CA000320EE75204E0E6CFEEFFE82EFAD7EF6A75
:109CB000E4EC1DF001EE6DF0020E016E086AF8C5CD
:109CC00021F0F7C520F0CFEC00F0EF6A04EEA5F02C
:109CD000260EF76E220EF66ED9EC02F011EE6DF044
:109CE000320EE75204E0E6CFEEFFE82EFAD7EF6A35
:109CF000E4EC1DF001EE6DF0020E016E086AFAC58B
:109D000021F0F9C520F0CFEC00F0EF6A04EEA5F0E9
:109D1000260EF76E320EF66ED9EC02F011EE6DF0F3
:109D2000320EE75204E0E6CFEEFFE82EFAD7EF6AF4
:109D3000E4EC1DF001EE6DF0020E016E086AFCC548
:109D400021F0FBC520F0CFEC00F0EF6A04EEA5F0A7
:109D5000260EF76E420EF66ED9EC02F011EE6DF0A3
:109D6000320EE75204E0E6CFEEFFE82EFAD7EF6AB4
:109D7000E4EC1DF001EE6DF0020E016E086AFEC506
:109D800021F0FDC520F0CFEC00F0EF6A04EEA5F065
:109D9000260EF76E520EF66ED9EC02F011EE6DF053
:109DA000320EE75204E0E6CFEEFFE82EFAD7EF6A74
:109DB000E4EC1DF001EE6DF0020E016E086A04C6BF
:109DC00021F003C620F0CFEC00F0EF6A04EEA5F01E
:109DD000260EF76E620EF66ED9EC02F011EE6DF003
:109DE000320EE75204E0E6CFEEFFE82EFAD7EF6A34
:109DF000E4EC1DF001EE6DF0020E016E086A06C67D
:109E000021F005C620F0CFEC00F0EF6A04EEA5F0DB
:109E1000260EF76E720EF66ED9EC02F011EE6DF0B2
:109E2000320EE75204E0E6CFEEFFE82EFAD7EF6AF3
:109E3000E4EC1DF001EE6DF0020E016E086A08C63A
:109E400021F007C620F0CFEC00F0EF6A04EEA5F099
:109E5000260EF76E820EF66ED9EC02F011EE6DF062
:109E6000320EE75204E0E6CFEEFFE82EFAD7EF6AB3
:109E7000E4EC1DF001EE6DF0020E016E086A0AC6F8
:109E800021F009C620F0CFEC00F0EF6A04EEA5F057
:109E9000260EF76E920EF66ED9EC02F011EE6DF012
:109EA000320EE75204E0E6CFEEFFE82EFAD7EF6A73
:109EB000E4EC1DF001EE6DF0020E016E086A0CC6B6
:109EC00021F00BC620F0CFEC00F0EF6A04EEA5F015
:109ED000260EF76EA20EF66ED9EC02F011EE6DF0C2
:109EE000320EE75204E0E6CFEEFFE82EFAD7EF6A33
:109EF000E4EC1DF0D8960501EEA9D8860001D8B68D
:109F00008DEF4FF001EEA0F0260EF76EB20EF66E5A
:109F1000D9EC02F0EF6A96EF4FF001EEA0F0260EBA
:109F2000F76EBC0EF66ED9EC02F0EF6A04EEA5F007
:109F3000260EF76EC80EF66ED9EC02F011EEA0F008
:109F4000140EE75204E0E6CFEEFFE82EFAD7EF6AF0
:109F5000E4EC1DF0D8960501EEABD8860001D8B62A
:109F6000BDEF4FF001EEA0F0260EF76ED60EF66EA6
:109F7000D9EC02F0EF6AC6EF4FF001EEA0F0260E2A
:109F8000F76EE00EF66ED9EC02F0EF6A04EEA5F083
:109F9000260EF76EEC0EF66ED9EC02F011EEA0F084
:109FA000140EE75204E0E6CFEEFFE82EFAD7EF6A90
:109FB000E4EC1DF0D8960501EEADD8860001D8B6C8
:109FC000EDEF4FF001EEA0F0260EF76EFA0EF66EF2
:109FD000D9EC02F0EF6AF6EF4FF001EEA0F0270E99
:109FE000F76E040EF66ED9EC02F0EF6A04EEA5F0FF
:109FF000270EF76E100EF66ED9EC02F011EEA0F0FF
:10A00000140EE75204E0E6CFEEFFE82EFAD7EF6A2F
:10A01000E4EC1DF0D8960501EEAFD8860001D8B665
:10A020001DEF50F001EEA0F0270EF76E1E0EF66E3B
:10A03000D9EC02F0EF6A26EF50F001EEA0F0270E07
:10A04000F76E280EF66ED9EC02F0EF6A04EEA5F07A
:10A05000270EF76E340EF66ED9EC02F011EEA0F07A
:10A06000140EE75204E0E6CFEEFFE82EFAD7EF6ACF
:10A07000E4EC1DF0D896060111A1D8860001D8B6EF
:10A080004DEF50F001EEA0F0270EF76E420EF66E87
:10A09000D9EC02F0EF6A56EF50F001EEA0F0270E77
:10A0A000F76E4C0EF66ED9EC02F0EF6A04EEA5F0F6
:10A0B000270EF76E580EF66ED9EC02F011EEA0F0F6
:10A0C000140EE75204E0E6CFEEFFE82EFAD7EF6A6F
:10A0D000E4EC1DF0D896060111A9D8860001D8B687
:10A0E0007FEF50F004EEA5F0270EF76E660EF66EC9
:10A0F000D9EC02F0EF6AE4EC1DF08AEF50F004EEC8
:10A10000A5F0270EF76E7C0EF66ED9EC02F0EF6A22
:10A11000E4EC1DF0D896060111ABD8860001D8B644
:10A120009FEF50F004EEA5F0270EF76E940EF66E3A
:10A13000D9EC02F0EF6AE4EC1DF0AAEF50F004EE67
:10A14000A5F0270EF76EAA0EF66ED9EC02F0EF6AB4
:10A15000E4EC1DF004EEA5F0270EF76EC20EF66ECD
:10A16000D9EC02F0020E016E05019151CCEC00F029
:10A17000EF6A0001E4EC1DF0050178530001D8A45A
:10A18000CBEF50F004EEA5F0270EF76ED20EF66E70
:10A19000D9EC02F0EF6A010E0501785D0001D8A448
:10A1A000DBEF50F004EEA5F0270EF76EEA0EF66E28
:10A1B000D9EC02F0EF6A020E0501785D0001D8A427
:10A1C000F8EF50F004EEA5F0280EF76E0E0EF66EC6
:10A1D000D9EC02F0020E016E7CC52FF07BC52EF08B
:10A1E0007AC52DF079C52CF0030EFEEC00F0EF6A75
:10A1F00001016C530001D8A409EF51F004EEA5F061
:10A20000280EF76E280EF66ED9EC02F0EF6AE4EC39
:10A210001DF0010E01016C5D0001D8A41BEF51F08F
:10A2200004EEA5F0280EF76E3C0EF66ED9EC02F0A7
:10A23000EF6AE4EC1DF001EE6DF0020E016E5BC5FD
:10A240002FF05AC52EF059C52DF058C52CF0030E2D
:10A25000FEEC00F0EF6A04EEA5F0280EF76E4E0E4D
:10A26000F66ED9EC02F011EE6DF0320EE75204E01A
:10A27000E6CFEEFFE82EFAD7EF6AE4EC1DF001EE30
:10A280006DF0020E016E6BC52FF06AC52EF069C528
:10A290002DF068C52CF0030EFEEC00F0EF6A04EE22
:10A2A000A5F0280EF76E5E0EF66ED9EC02F011EEF8
:10A2B0006DF0320EE75204E0E6CFEEFFE82EFAD75B
:10A2C000EF6AE4EC1DF001EE6DF0020E016E4BC57D
:10A2D0002FF04AC52EF049C52DF048C52CF0030ECD
:10A2E000FEEC00F0EF6A04EEA5F0280EF76E6E0E9D
:10A2F000F66ED9EC02F011EE6DF0320EE75204E08A
:10A30000E6CFEEFFE82EFAD7EF6AE4EC1DF001EE9F
:10A310006DF0020E016E5FC52FF05EC52EF05DC5BB
:10A320002DF05CC52CF0030EFEEC00F0EF6A04EE9D
:10A33000A5F0280EF76E7E0EF66ED9EC02F011EE47
:10A340006DF0320EE75204E0E6CFEEFFE82EFAD7CA
:10A35000EF6AE4EC1DF001EE6DF0020E016E6FC5C8
:10A360002FF06EC52EF06DC52DF06CC52CF0030ED0
:10A37000FEEC00F0EF6A04EEA5F0280EF76E8E0EEC
:10A38000F66ED9EC02F011EE6DF0320EE75204E0F9
:10A39000E6CFEEFFE82EFAD7EF6AE4EC1DF001EE0F
:10A3A0006DF0020E016E4FC52FF04EC52EF04DC55B
:10A3B0002DF04CC52CF0030EFEEC00F0EF6A04EE1D
:10A3C000A5F0280EF76E9E0EF66ED9EC02F011EE97
:10A3D0006DF0320EE75204E0E6CFEEFFE82EFAD73A
:10A3E000EF6AE4EC1DF001EE6DF0020E016E63C544
:10A3F0002FF062C52EF061C52DF060C52CF0030E64
:10A40000FEEC00F0EF6A04EEA5F0280EF76EAE0E3B
:10A41000F66ED9EC02F011EE6DF0320EE75204E068
:10A42000E6CFEEFFE82EFAD7EF6AE4EC1DF001EE7E
:10A430006DF0020E016E73C52FF072C52EF071C55E
:10A440002DF070C52CF0030EFEEC00F0EF6A04EE68
:10A45000A5F0280EF76EBE0EF66ED9EC02F011EEE6
:10A460006DF0320EE75204E0E6CFEEFFE82EFAD7A9
:10A47000EF6AE4EC1DF001EE6DF0020E016E53C5C3
:10A480002FF052C52EF051C52DF050C52CF0030E03
:10A49000FEEC00F0EF6A04EEA5F0280EF76ECE0E8B
:10A4A000F66ED9EC02F011EE6DF0320EE75204E0D8
:10A4B000E6CFEEFFE82EFAD7EF6AE4EC1DF001EEEE
:10A4C0006DF0020E016E67C52FF066C52EF065C5F2
:10A4D0002DF064C52CF0030EFEEC00F0EF6A04EEE4
:10A4E000A5F0280EF76EDE0EF66ED9EC02F011EE36
:10A4F0006DF0320EE75204E0E6CFEEFFE82EFAD719
:10A50000EF6AE4EC1DF001EE6DF0020E016E77C50E
:10A510002FF076C52EF075C52DF074C52CF0030E06
:10A52000FEEC00F0EF6A04EEA5F0280EF76EEE0EDA
:10A53000F66ED9EC02F011EE6DF0320EE75204E047
:10A54000E6CFEEFFE82EFAD7EF6AE4EC1DF001EE5D
:10A550006DF0020E016E57C52FF056C52EF055C591
:10A560002DF054C52CF0030EFEEC00F0EF6A04EE63
:10A57000A5F0280EF76EFE0EF66ED9EC02F011EE85
:10A580006DF0320EE75204E0E6CFEEFFE82EFAD788
:10A59000EF6AE4EC1DF0050126530001D8A4DCEFBE
:10A5A00052F004EEA5F0290EF76E0E0EF66ED9EC01
:10A5B00002F0EF6AE4EC1DF0010E0501265D0001DA
:10A5C000D8A4EEEF52F004EEA5F0290EF76E240E9B
:10A5D000F66ED9EC02F0EF6AE4EC1DF01200DAEC52
:04A5E0004BF012002A
:020000040030CA
:03000100861A0F4D
:020005008181F7
:060008000FC00FE00F40E5
:00000001FF
